:020000040000FA
:3C000000FFFF627515FFFFFFFFFFFFFFFFFFFFFFFFFFFFFFFFFFFFFFFFFFFFFFFFFFFFFFFFFFFFFFFFFFFFFFFFFFFFFFFFFFFFFFFFFFFFFFFFFFFFFFFFFFFFFF11
:3C003C00000000000000000000000000000000000008000000080008000000000000000000000000000000000000000000000000000000000000000000009EFED4
:3C0078000000000000000000000000000000000004800400048000800000040000000000000000000000040000000000000000000000000000000000000096FE24
:3C00B40000000000000000000000048000000000000000000000000004000000000000000000040004800000048000800400048000800480040004800000DAFE10
:3C00F0000000048004800480048000800480048014A8148814A804A004801488048004800480008004801488048004800480048004000080048004800000F8FEA6
:3C012C0000000480048004800480048004800480048804800488248004800480048004800480048024800480348024800480248004800488048004900000B6FE1F
:3C016800000004000480000000000480000000000480040004800080040004000000000000000400048004000480008004000480008004800400048000001AFEFF
:3C01A4000000008000000480048004800480048004800480048004800480048004800480048004800480048004800480048004800480048004800480000056FE67
:3C01E00000000080000004800480048004800480304030803040042034803080048004800480048004A0308024A004A034800CA8048034C00C880CA8000072FF52
:3C021C0000000000000000000000000000000000000000000000000000000000000000000000000000000080160000000000000000000000000000C1160037FF03
:3C0258000000000000000000000000000000000000000000000000000000000000000000000000000000000006000000000000000000000000000000000018FE4E
:3C0294000000000000000000000000000000000000000000000000000000000000000000000000000000008000000000000000000000000000000080060070FEBA
:3C02D00002000000000000000000000000000000000000000000000000000000000000000000000000000080000800000000000000000000000000800004EFFFF6
:3C030C000200000000000000000000000000000000000000000000000000000000000000000000000000008000000000000000000000000000000084003001FE80
:3C0348000200000000000000000000000000000000000000000000000000000000000000000000000000000000000000000000000000000000000000060049FF29
:3C0384000000000000000000000000000000000000000000000000000000000000000000000000000000008006000000000000000100000000000080040055FFDE
:3C03C00000000000000000000000000000000000000000000000000000000000000000000000000000000000060000000000008000000080010000408A007BFEB7
:3C03FC0000000000000000000000000000000000000000000000000000000000000000000000000000000082020000000000000000000000000000C1160012FE5A
:3C043800000000000000000000000000000000000000000000000000000000000000000000000000000000000200000000000000000000000000000000001CFE6C
:3C0474000000000000000000000000000000000000000000000000000000000000000000000000000000008002000000000000000000000000000080060072FED4
:3C04B000020000000000000000000000000000000000000000000000000000000000000000000000000000C02A000000000000000000000000000080000409FF98
:3C04EC0002000000000000000000000000000000000000000000000000000000000000000000000000000080080000000000000000000000000000C200006DFF1C
:3C0528000000000000000000000000000000000000000000000000000000000000000000000000000000000000000000000000000000000000000000060078FE1B
:3C0564000200000000000000000000000000000000000000000000000000000000000000000000000000008006000000000000000000010000000080040065FEEB
:3C05A00002000000000000000000000000000000000000000000000000000000000000000000000000000000060800000000000000800000000000000A04CBFFB7
:3C05DC00000000000000000000000000000000000000000000000000000000000000000000000000000000C4060000000000000000000000000000C1120067FFE0
:3C061800000000000000000000000000000000000000000000000000000000000000000000000000000000000600000000000000000000000000000002003AFE66
:3C0654000000000000000000000000000000000000000000000000000000000000000000000000000000008006000000000000000000000000000080020032FE32
:3C0690000200000000000000000000000000000000000000000000000000000000000000000000000000008006000000000000000000000000000080020443FFDE
:3C06CC0002000000000000000000000000000000000000000000000000000000000000000000000000000080000000000000000000000000000000A40C508BFEE7
:3C070800020000000000000000000000000000000000000000000000000000000000000000000000000000000000000000000000000000000000000002000DFFA5
:3C0744000000000000000000000000000000000000000000000000000000000000000000000000000000008000000000000000000000000000000080000007FF73
:3C078000000000000000000000000000000000000000000000000000000000000000000000000000000000000000000000000000000000000000000026006BFFAD
:3C07BC00000000000000000000000000000000000000000000000000000000000000000000000000000000C40E00000000000000000000A4160000C11600D7FFC8
:3C07F800000000000000000000000000000000000000000000000000000000000000000000000000000000000600000000000000000000000200000000001AFEA5
:3C08340000000000000000000000000000000000000000000000000000000000000000000000000000000080060000000000000000000080000000800600FEFE00
:3C08700002000000000000000000000000000000000000000000000000000000000000000000000000000080260000000000000000000080220000800004EBFF94
:3C08AC00020000000000000000000000000000000000000000000000000000000000000000000000000000801400000000000000000000C1000080C0001027FE44
:3C08E800020000000000000000000000000000000000000000000000000000000000000000000000000000000200000000000000000000000000000006004BFF80
:3C09240000000000000000000000000000000000000000000000000000000000000000000000000000000080060000000000000000000080060000800400CBFF3D
:3C096000000000000000000000000000000000000000000000000000000000000000000000000000000000000608000000000000008001801702000012449BFE44
:3C099C000000000000000000000000000000408006C1868046C006A206A8020000000000000000824680068216080608068216C1128806A4060000420600EFFE5A
:3C09D8000000000000000000000000000000000006000600060006000600020000000000000000000600060006000600060006000200060002000000060078FE19
:3C0A140000000000000000000000000000000080068006800680068002800200000000000000008000800680008002800280008002800280000000800200DEFE9E
:3C0A5000020000000000000000000000000000A0368036C0368036803280320000000000000000C010A836C000C132C032C0008202C4528032000080320095FE28
:3C0A8C00020000000000000000000000000000A8008210A80082108000820C00000000000000008004A8008004800080008084A0048000C10800008020000DFE5E
:3C0AC800020000000000000000000000000000000000000000000000000002000000000000000000020000000200000000000200020000000000000000000DFFDA
:3C0B0400000000000000000000000000000000800280028002800380028006000000000000000080048002800480028002800480018000800600008002008FFEFC
:3C0B4000000000000000000000000000000000000842000808C200080C42820000000000000000003200080232000C020C02328036008800060800000C2263FFED
:3C0B7C00000000000000000000000000000000000000000000000000000000000000000000000000000000900E0000000000000000000000000000100E0066FF1C
:3C0BB800000000000000000000000000000000000000000000000000000000000000000000000000000000000600000000000000000000000000000006007EFE79
:3C0BF4000000000000000000000000000000000000000000000000000000000000000000000000000000008000000000000000000000000000000080040052FE71
:3C0C3000020000000000000000000000000000000000000000000000000000000000000000000000000000A0060400000000000000000000000000A0240021FFF8
:3C0C6C000200000000000000000000000000000000000000000000000000000000000000000000000000008200000000000000000000000000000080000007FF42
:3C0CA800020000000000000000000000000000000000000000000000000000000000000000000000000000000000000000000000000000000000000000003EFED2
:3C0CE4000000000000000000000000000000000000000000000000000000000000000000000000000000008000000000000000000000000001000080040053FE7E
:3C0D200000000000000000000000000000000000000000000000000000000000000000000000000000000040060000000000000000000080000000000A024FFF77
:3C0D5C0000000000000000000000000000000000000000000000000000000000000000000000000000A216B00E00000000000000000000000000000416001CFFB0
:3C0D9800000000000000000000000000000000000000000000000000000000000000000000000000000002000600000000000000000000000000000006005CFEB7
:3C0DD4000000000000000000000000000000000000000000000000000000000000000000000000000000008000000000000000000000000000000080020034FEAF
:3C0E100002000000000000000000000000000000000000000000000000000000000000000000000000800282860000000000000000000000000000A0021021FE49
:3C0E4C00020000000000000000000000000000000000000000000000000000000000000000000000002800820000000000000000000000000000008000002FFF10
:3C0E8800000000000000000000000000000000000000000000000000000000000000000000000000000000000000000000000000000000000000000000001EFE12
:3C0EC4000200000000000000000000000000000000000000000000000000000000000000000000000080008000000000000000000000000000000080020085FFEA
:3C0F000002000000000000000000000000000000000000000080010000000000000000000000000000000E42060000000000008001000080010000000C0257FF76
:3C0F3C0000000000000000000000000000000000000000000000000000000000000000000000000000000090060000000000000000000000000000040E007AFF58
:3C0F78000000000000000000000000000000000000000000000000000000000000000000000000000000000002000000000000800000000000000000060072FE45
:3C0FB40000000000000000000000000000000000000000000000000000000000000000000000000000000000020000000000000000000000000000800200BEFEC1
:3C0FF000020000000000000000000000000000000000000000000000000000000000000000000000000000A0120200000000000000000000000000C0021057FEE8
:3C102C00020000000000000000000000000000000000000000000000000000000000000000000000000000021000000000000000000000000000008000009FFF56
:3C106800000000000000000000000000000000000000000000000000000000000000000000000000000000000000000000000000000000000000000000001EFE30
:3C10A4000200000000000000000000000000000000000000000000000000000000000000000000000000008000000000000000000000000000000080020005FF08
:3C10E00002000000000000000000000000000000000000000000000000000000000000000000000000000040040800000000008000000080010000000C029BFEDE
:3C111C00000000000000000000000000000000000000000000000000000000000000000000000000008816B006000000000000000000000000000002060028FE15
:3C1158000000000000000000000000000000000000000000000000000000000000000000000000000000020002000000000000000000000000000000060058FEFB
:3C11940000000000000000000000000000000000000000000000000000000000000000000000000000000600020000000000000000000000000000800200D8FEBF
:3C11D00002000000000000000000000000000000000000000000000000000000000000000000000000C00084120400000000000000000000000000C00A101BFE94
:3C120C0002000000000000000000000000000000000000000000000000000000000000000000000000280002100000000000000000000000000000800000B7FF34
:3C124800000000000000000000000000000000000000000000000000000000000000000000000000000000000000000000000000000000000000000000001EFE4E
:3C12840002000000000000000000000000000000000000000000000000000000000000000000000000800480000000000100000001000000000000800200D1FED5
:3C12C00002000000000000000000000000000000000000000000008001000000008001000000000000800942040800800000008000000000000000000C02ABFE60
:3C12FC00000000000000000000000000000000000088160000881600000000000000000000000000008886800688168816000008068810081688964006003EFF45
:3C1338000000000000000000000000000000000000000600000006000000008000000000000000000000060002000200020000000600060006000600060090FE35
:3C137400000000000000000000000000000000000080000000800000000000000000000000000000008004000480068006000080048004800480008006003EFEDB
:3C13B0000200000000000000000000000000000000C0440000C0040400000000000000000000000000C00CC428C006C4060400C034C006C424C08680080221FE56
:3C13EC000200000000000000000000000000000000821000008210000000000000000000000000000080000290C008C4080000800082088000820088000065FE02
:3C14280000800080008000800080008000800080008000800080008000800080008000800080008000800080008000800080008000800480008000800600BCFEC4
:3C146400020000000000000000000000000000000000060000000600000000000000000000000000000004000400000000000000040000000400010001005DFED1
:3C14A00002000000000000000000000000000000004006080040068801000080000000000080010000000A4202080401040100800B4200010AC206C00000AFFF82
:3C14DC00000000000000000000000000000000000000000000000000000000000000000000000000000000000008000800000008000000080000000800009EFE10
:3C151800000000000000000000000000000000080008000800080008000800000000000000000008000800080020002000080020000800200008002000003CFE5D
:3C155400000000000000000000000000000000000000000000000000000000000000000000000000000000000000000000000000000000000000000000001EFE3F
:3C159000000000000000000000000000000000000000000000000000000000000000000000000000000000000000000000000000000000000000000000001EFE03
:3C15CC00000000000000000000000000000000000000000000000000000000000000000000000000000000000000000000000000000000000000000000001EFEC7
:3C160800000000000000000000000000000000000000000000000000000000000000000000000000000000000000000000000000000000000000200002001EFE68
:3C16440000000000000000000000000000000000000000000000000000000000000000000000000008000000000000200220000000200020010000000040E8FFB8
:3C16800000000000000000000000000000000000000000000000000000000000000000000000000000000000000000000000000005000000000008080000C6FE55
:3C16BC00000000000000000000000000000000000000000000000000000000000000000000000000002000000000000000000000020000000000000000001EFEB4
:3C16F8000000000000000000000000000000000000000000000001000000000000000400000000000002002000400000000010000000000000000220002058FFA6
:3C173400000000000000000000000000000000000040004000400040000000400000000000000000000000400000000000000000000004000000000000005EFE99
:3C1770000000000000000000000000000000000000080000000800020008000000000000000000080000000800000008000800000008010004080000001038FEA8
:3C17AC00000000000000000000000000000000000000000000000000000000000000000000000000000000000000000000000000000000000000000000001EFEE5
:3C17E800000000000000000000000000000010000000000000000000000000000000000000000400000002002200000100010001000000010000000100000AFE80
:3C182400000000000000000000000000000000000000000000000000000000000400000000000000000040000000000000000000000000000000000040001AFEEC
:3C18600000000000000000000000000000000000000000000000000006000000000000000000000000000008001200100000000000000000000200000410BAFE4E
:3C189C00000000000000000000000000000000000000000000000000000000000000000000000000000000000000000000000000000000000000000000001EFEF4
:3C18D800000000000000000000000000000000000000000000000000000000000000000000000000000000000000000000000000000000000000000440001EFE74
:3C191400000000000000000000000000000000000000000000000000000000000000000000000000000000000000000000000000000000000000000000001EFE7B
:3C195000000000000000000000000000000000000000000000000000000000000000000000000000000000000000000000000000000000000000000000001EFE3F
:3C198C00000000000000000000000000000000000001000000000000000000000000000000000000000000001000000000000000000000000000000000000EFF01
:3C19C800000000000000000000000000000000000000000000000000000000000000000000000000000000000000000000000000000000000000000000001EFEC7
:3C1A0400000000000000000000000000000000000000000000000000000000000000000000000000000000000000000000000000000000000000000000001EFE8A
:3C1A4000000000000000000000000000000000000000000000000000000000000000000000000000000000040000000000000000000000001000000000004EFE0A
:3C1A7C00000000000000000000000000000000000000000000000000000000000000000000000000000000000000000000000000000000000000000000001EFE12
:3C1AB800000000000000000000000000000000000000000000000000000000000000000000000000000000008000000000000000080000000000000000001EFE4E
:3C1AF4000000000000000000000000000000000000000000000000000000400000000000000000000010000000000000000000000008100000000000000012FF3D
:3C1B30000000000000000000000000000000000000000000000000000000000000000000000000000000000000000000000000042000000000000000000078FEDF
:3C1B6C00000000000000000000000000000000000000000004000000000000000000000000000000000000040000000000000000000000000000000000001AFE1D
:3C1BA8000000000000000000000000000000008000000080000020800080000000000000000000000080000000800100000000000000000020000100000016FEAB
:3C1BE400000000000000000000000000000000000000220000000000000000000000000000000000000000000000000000000002000000020001005200004CFF01
:3C1C2000000000000000000000000000000000000000000000000000000000000000000000000000000000000000000000000000000000000000000000001EFE6C
:3C1C5C00000000000000000000000000000000000000000000000020000000000000000000000000000020000000000000000000000000000000000000001EFEF0
:3C1C98000000000000000000000000000000000000000000000000000000000000000000000000000000000008000000000000000000200000000000000014FED6
:3C1CD400000000000000000000000000000000000000000000000000000000000000000000000000000000000000000000000000000000000000000000001EFEB8
:3C1D10000000000000000000000000000000000000000000000000000000000000000000000000000000000808010000000000000000000000000000000096FFF1
:3C1D4C00000000000000000000000000000000000000000000000000000000000000000000000000000000000000000000000000000000000000000000000FFF4D
:3C1D8800000000000000000000000000000000000000000000000000000000000000000000000000000000000000000000000000000000000000000000001EFE03
:3C1DC400000000000000000000000000000000000000000000000000000000000000000000000000000000000000000000000000000000000000000000001EFEC7
:3C1E0000020000000000000000000000000000000000000000000000000000000000000000000000000000000000000000000000000000000000000000003EFE68
:3C1E3C00020000000000000000000000000000000000000000000000000000000000000000000000000000000000000000000000000000000000000000002FFF3A
:3C1E7800000000000000000000000000000000000000000000000000000000000000000000000000000000000000000000000000000000000000000000000FFF20
:3C1EB400020000000000000000000000000000000000000000000000000000000000000000000000000000000000000000000000000000000000000000003EFEB4
:3C1EF000020000000000000000000000000000000000000000000000000000000000000000000000000000000000000000000000000000000000000000003EFE78
:3C1F2C00020000000000000000000000000000000000000000000000000000000000000000000000000000000000000000000000000000000000000000003EFE3B
:3C1F6800000000000000000000000000000000000000000000000000000000000000000000000000000000000000000000000000000000000000000000001EFE21
:3C1FA400000000000000000000000000000000000000000000000000000000000000000000000000000000000000000000000000000000000000000000001EFEE5
:3C1FE000020000000000000000000000000000000000000000000000000000000000000000000000000000000000000000000000000000000000000000002FFF95
:3C201C00020000000000000000000000000000000000000000000000000000000000000000000000000000000000000000000000000000000000000000002FFF58
:3C205800020000000000000000000000000000000000000000000000000000000000000000000000000000000000000000000000000000000000000000002FFF1C
:3C209400020000000000000000000000000000000000000000000000000000000000000000000000000000000000000000000000000000000000000000003EFED2
:3C20D000020000000000000000000000000000000000000000000000000000000000000000000000000000000000000000000000000000000000000000003EFE96
:3C210C00000000000000000000000000000000000000000000000000000000000000000000000000000000000000000000000000000000000000000000001EFE7B
:3C214800000000000000000000000000000000000000000000000000000000000000000000000000000000000000000000000000000000000000000000001EFE3F
:3C218400000000000000000000000000000000000000000000000000000000000000000000000000000000000000000000000000000000000000000000001EFE03
:3C21C000020000000000000000000000000000000000000000000000000000000000000000000000000000000000000000000000000000000000000000002FFFB3
:3C21FC00020000000000000000000000000000000000000000000000000000000000000000000000000000000000000000000000000000000000000000002FFF77
:3C223800000000000000000000000000000000000000000000000000000000000000000000000000000000000000000000000000000000000000000000001EFE4E
:3C227400020000000000000000000000000000000000000000000000000000000000000000000000000000000000000000000000000000000000000000002FFFFE
:3C22B000020000000000000000000000000000000000000000000000000000000000000000000000000000000000000000000000000000000000000000002FFFC2
:3C22EC00020000000000000000000000000000000000000000000000000000000000000000000000000000000000000000000000000000000000000000003EFE78
:3C232800000000000000000000000000000000000000000000000000000000000000000000000000000000000000000000000000000000000000000000001EFE5D
:3C236400000000000000000000000000000000000000000000000000000000000000000000000000000000000000000000000000000000000000000000001EFE21
:3C23A000020000000000000000000000000000000000000000000000000000000000000000000000000000000000000000000000000000000000000000002FFFD1
:3C23DC00020000000000000000000000000000000000000000000000000000000000000000000000000000000000000000000000000000000000000000002FFF95
:3C241800020000000000000000000000000000000000000000000000000000000000000000000000000000000000000000000000000000000000000000003EFE4A
:3C245400020000000000000000000000000000000000000000000000000000000000000000000000000000000000000000000000000000000000000000002FFF1C
:3C249000020000000000000000000000000000000000000000000000000000000000000000000000000000000000000000000000000000000000000000002FFFE0
:3C24CC00000000000000000000000000000000000000000000000000000000000000000000000000000000000000000000000000000000000000000000000FFFC6
:3C250800000000000000000000000000000000000000000000000000000000000000000000000000000000000000000000000000000000000000000000001EFE7B
:3C254400000000000000000000000000000000000000000000000000000000000000000000000000000000000000000000000000000000000000000000001EFE3F
:3C258000020000000000000000000000000000000000000000000000000000000000000000000000000000000000000000000000000000000000000000003EFEE1
:3C25BC00020000000000000000000000000000000000000000000000000000000000000000000000000000000000000000000000000000000000000000002FFFB3
:3C25F800000000000000000000000000000000000000000000000000000000000000000000000000000000000000000000000000000000000000000000000FFF99
:3C263400020000000000000000000000000000000000000000000000000000000000000000000000000000000000000000000000000000000000000000003EFE2C
:3C267000020000000000000000000000000000000000000000000000000000000000000000000000000000000000000000000000000000000000000000003EFEF0
:3C26AC00000000000000000000000000000000000000000000000000000000000000000000000000000000000000000000000000000000000000000000001EFED6
:3C26E800000000000000000000000000000000000000000000000000000000000000000000000000000000000000000000000000000000000000000000001EFE9A
:3C272400000000000000000000000000000000000000000000000000000000000000000000000000000000000000000000000000000000000000000000001EFE5D
:3C276000020000000000000000000000000000000000000000000000000000000000000000000000000000000000000000000000000000000000000000002FFF0D
:3C279C00020000000000000000000000000000000000000000000000000000000000000000000000000000000000000000000000000000000000000000002FFFD1
:3C27D800000000000000000000000000000000000000000000000000000000000000000000000000000000000000000000000000000000000000000000001EFEA9
:3C281400020000000000000000000000000000000000000000000000000000000000000000000000000000000000000000000000000000000000000000002FFF58
:3C285000020000000000000000000000000000000000000000000000000000000000000000000000000000000000000000000000000000000000000000002FFF1C
:3C288C00000000000000000000000000000000000000000000000000000000000000000000000000000000000000000000000000000000000000000000000FFF02
:3C28C800000000000000000000000000000000000000000000000000000000000000000000000000000000000000000000000000000000000000000000001EFEB8
:3C290400000000000000000000000000000000000000000000000000000000000000000000000000000000000000000000000000000000000000000000001EFE7B
:3C294000020000000000000000000000000000000000000000000000000000000000000000000000000000000000000000000000000000000000000000003EFE1D
:3C297C00020000000000000000000000000000000000000000000000000000000000000000000000000000000000000000000000000000000000000000002FFFEF
:3C29B800000000000000000000000000000000000000000000000000000000000000000000000000000000000000000000000000000000000000000000000FFFD5
:3C29F400020000000000000000000000000000000000000000000000000000000000000000000000000000000000000000000000000000000000000000003EFE69
:3C2A3000020000000000000000000000000000000000000000000000000000000000000000000000000000000000000000000000000000000000000000003EFE2C
:3C2A6C00000000000000000000000000000000000000000000000000000000000000000000000000000000000000000000000000000000000000000000000FFF20
:3C2AA800000000000000000000000000000000000000000000000000000000000000000000000000000000000000000000000000000000000000000000001EFED6
:3C2AE400000000000000000000000000000000000000000000000000000000000000000000000000000000000000000000000000000000000000000000001EFE9A
:3C2B2000020000000000000000000000000000000000000000000000000000000000000000000000000000000000000000000000000000000000000000003EFE3B
:3C2B5C00020000000000000000000000000000000000000000000000000000000000000000000000000000000000000000000000000000000000000000002FFF0D
:3C2B9800000000000000000000000000000000000000000000000000000000000000000000000000000000000000000000000000000000000000000000000FFFF3
:3C2BD400020000000000000000000000000000000000000000000000000000000000000000000000000000000000000000000000000000000000000000003EFE87
:3C2C1000020000000000000000000000000000000000000000000000000000000000000000000000000000000000000000000000000000000000000000003EFE4A
:3C2C4C00000000000000000000000000000000000000000000000000000000000000000000000000000000000000000000000000000000000000000000001EFE30
:3C2C8800000000000000000000000000000000000000000000000000000000000000000000000000000000000000000000000000000000000000000000001EFEF4
:3C2CC400000000000000000000000000000000000000000000000000000000000000000000000000000000000000000000000000000000000000000000001EFEB8
:3C2D0000020000000000000000000000000000000000000000000000000000000000000000000000000000000000000000000000000000000000000000002FFF67
:3C2D3C00020000000000000000000000000000000000000000000000000000000000000000000000000000000000000000000000000000000000000000002FFF2B
:3C2D7800020000000000000000000000000000000000000000000000000000000000000000000000000000000000000000000000000000000000000000003EFEE1
:3C2DB400000000000000000000000000000000000000000000000000000000000000000000000000000000000000000000000000000000000000000000000FFFD5
:3C2DF000000000000000000000000000000000000000000000000000000000000000000000000000000000000000000000000000000000000000000000000FFF99
:3C2E2C00000000000000000000000000000000000000000000000000000000000000000000000000000000000000000000000000000000000000000000000FFF5C
:3C2E6800000000000000000000000000000000000000000000000000000000000000000000000000000000000000000000000000000000000000000000001EFE12
:3C2EA400000000000000000000000000000000000000000000000000000000000000000000000000000000000000000000000000000000000000000000001EFED6
:3C2EE000020000000000000000000000000000000000000000000000000000000000000000000000000000000000000000000000000000000000000000003EFE78
:3C2F1C00020000000000000000000000000000000000000000000000000000000000000000000000000000000000000000000000000000000000000000002FFF49
:3C2F5800008000800080008000800080008000800080008000800080008000800080008000800080008000800080008000800080008000800080008000008FFFAF
:3C2F9400020000000000000000000000000000000000000000000000000000000000000000000000000000000000000000000000000000000000000000003EFEC3
:3C2FD000020000000000000000000000000000000000000000000000000000000000000000000000000000000000000000000000000000000000000000003EFE87
:3C300C00000000000000000000000000000000000000000000000000000000000000000000000000000000000000000000000000000000000000000000001EFE6C
:3C304800000000000000000000000000000000000000000000000000000000000000000000000000000000000000000000000000000000000000000000001EFE30
:3C308400000000000000000000000000000000000000000000000000000000000000000000000000000000000000000000000000000000000000000000001EFEF4
:3C30C000000000000000000000000000000000000000000000000000000000000000000000000000000000000000000000000000000000000000000000001EFEB8
:3C30FC00000000000000000000000000000000000000000000000000000000000000000000000000000000000000000000000000000000000000000000001EFE7C
:3C313800000000000000000000000000000000000000000000000000000000000000000000000000000000000000000000000000000000000000000000001EFE3F
:3C317400000000000000000000000000000000000000000000000000000000000000000000000000000000000000000000000000000000000000000000001EFE03
:3C31B000000000000000000000000000000000000000000000000000000000000000000000000000000000000000000000000000000000000000000000001EFEC7
:3C31EC00000000000000000000000000000000000000000000000000000000000000000000000000000000000000000000000000000000000000000000001EFE8B
:3C322800000000000000000000000000000000000000000000000000000000000000000000000000000000000000000000000000000000000000000000001EFE4E
:3C326400000000000000000000000000000000000000000000000000000000000000000000000000000000000000000000000000000000000000000000001EFE12
:3C32A000000000000000000000000000000000000000000000000000000000000000000000000000000000000000000000000000000000000000000000001EFED6
:3C32DC00000000000000000000000000000000000000000000000000000000000000000000000000000000000000000000000000000000000000000000001EFE9A
:3C331800000000000000000000000000000000000000000000000000000000000000000000000000000000000000000000000000000000000000000000001EFE5D
:3C335400000000000000000000000000000000000000000000000000000000000000000000000000000000000000000000000000000000000000000000001EFE21
:3C339000000000000000000000000000000000000000000000000000000000000000000000000000000000000000000000000000000000000000000000001EFEE5
:3C33CC00000000000000000000000000000000000000000000000000000000000000000000000000000000000000000000000000000000000000000000001EFEA9
:3C340800000000000000000000000000000000000000000000000000000000000000000000000000000000000000000000000000000000000000000000001EFE6C
:3C344400000000000000000000000000000000000000000000000000000000000000000000000000000000000000000000000000000000000000000000001EFE30
:3C348000000000000000000000000000000000000000000000000000000000000000000000000000000000000000000000000000000000000000000000001EFEF4
:3C34BC00000000000000000000000000000000000000000000000000000000000000000000000000000000000000000000000000000000000000000000001EFEB8
:3C34F800000000000000000000000000000000000000000000000000000000000000000000000000000000000000000000000000000000000000000000001EFE7C
:3C353400000000000000000000000000000000000000000000000000000000000000000000000000000000000000000000000000000000000000000000001EFE3F
:3C357000000000000000000000000000000000000000000000000000000000000000000000000000000000000000000000000000000000000000000000001EFE03
:3C35AC00000000000000000000000000000000000000000000000000000000000000000000000000000000000000000000000000000000000000000000001EFEC7
:3C35E800000000000000000000000000000000000000000000000000000000000000000000000000000000000000000000000000000000000000000000001EFE8B
:3C362400000000000000000000000000000000000000000000000000000000000000000000000000000000000000000000000000000000000000000000001EFE4E
:3C366000000000000000000000000000000000000000000000000000000000000000000000000000000000000000000000000000000000000000000000001EFE12
:3C369C00000000000000000000000000000000000000000000000000000000000000000000000000000000000000000000000000000000000000000000001EFED6
:3C36D800000000000000000000000000000000000000000000000000000000000000000000000000000000000000000000000000000000000000000000001EFE9A
:3C371400000000000000000000000000000000000000000000000000000000000000000000000000000000000000000000000000000000000000000000001EFE5D
:3C375000000000000000000000000000000000000000000000000000000000000000000000000000000000000000000000000000000000000000000000001EFE21
:3C378C00000000000000000000000000000000000000000000000000000000000000000000000000000000000000000000000000000000000000000000001EFEE5
:3C37C800000000000000000000000000000000000000000000000000000000000000000000000000000000000000000000000000000000000000000000001EFEA9
:3C380400000000000000000000000000000000000000000000000000000000000000000000000000000000000000000000000000000000000000000000001EFE6C
:3C384000000000000000000000000000000000000000000000000000000000000000000000000000000000000000000000000000000000000000000000001EFE30
:3C387C00000000000000000000000000000000000000000000000000000000000000000000000000000000000000000000000000000000000000000000001EFEF4
:3C38B800000000000000000000000000000000000000000000000000000000000000000000000000000000000000000000000000000000000000000000001EFEB8
:3C38F400000000000000000000000000000000000000000000000000000000000000000000000000000000000000000000000000000000000000000000001EFE7C
:3C393000020000000000000000000000000000000000000000000000000000000000000000000000000000000000000000000000000000000000000000002FFF2B
:3C396C00020000000000000000000000000000000000000000000000000000000000000000000000000000000000000000000000000000000000000000002FFFEF
:3C39A800000000000000000000000000000000000000000000000000000000000000000000000000000000000000000000000000000000000000000000001EFEC7
:3C39E400020000000000000000000000000000000000000000000000000000000000000000000000000000000000000000000000000000000000000000002FFF77
:3C3A2000020000000000000000000000000000000000000000000000000000000000000000000000000000000000000000000000000000000000000000002FFF3A
:3C3A5C00000000000000000000000000000000000000000000000000000000000000000000000000000000000000000000000000000000000000000000001EFE12
:3C3A9800000000000000000000000000000000000000000000000000000000000000000000000000000000000000000000000000000000000000000000001EFED6
:3C3AD400000000000000000000000000000000000000000000000000000000000000000000000000000000000000000000000000000000000000000000001EFE9A
:3C3B1000020000000000000000000000000000000000000000000000000000000000000000000000000000000000000000000000000000000000000000002FFF49
:3C3B4C00020000000000000000000000000000000000000000000000000000000000000000000000000000000000000000000000000000000000000000002FFF0D
:3C3B8800020000000000000000000000000000000000000000000000000000000000000000000000000000000000000000000000000000000000000000003EFEC3
:3C3BC400000000000000000000000000000000000000000000000000000000000000000000000000000000000000000000000000000000000000000000000FFFB7
:3C3C0000000000000000000000000000000000000000000000000000000000000000000000000000000000000000000000000000000000000000000000000FFF7A
:3C3C3C00000000000000000000000000000000000000000000000000000000000000000000000000000000000000000000000000000000000000000000000FFF3E
:3C3C7800000000000000000000000000000000000000000000000000000000000000000000000000000000000000000000000000000000000000000000001EFEF4
:3C3CB400000000000000000000000000000000000000000000000000000000000000000000000000000000000000000000000000000000000000000000001EFEB8
:3C3CF000020000000000000000000000000000000000000000000000000000000000000000000000000000000000000000000000000000000000000000002FFF68
:3C3D2C00020000000000000000000000000000000000000000000000000000000000000000000000000000000000000000000000000000000000000000002FFF2B
:3C3D6800020000000000000000000000000000000000000000000000000000000000000000000000000000000000000000000000000000000000000000002FFFEF
:3C3DA400000000000000000000000000000000000000000000000000000000000000000000000000000000000000000000000000000000000000000000000FFFD5
:3C3DE000000000000000000000000000000000000000000000000000000000000000000000000000000000000000000000000000000000000000000000000FFF99
:3C3E1C00000000000000000000000000000000000000000000000000000000000000000000000000000000000000000000000000000000000000000000000FFF5C
:3C3E5800000000000000000000000000000000000000000000000000000000000000000000000000000000000000000000000000000000000000000000001EFE12
:3C3E9400000000000000000000000000000000000000000000000000000000000000000000000000000000000000000000000000000000000000000000001EFED6
:3C3ED000020000000000000000000000000000000000000000000000000000000000000000000000000000000000000000000000000000000000000000002FFF86
:3C3F0C00020000000000000000000000000000000000000000000000000000000000000000000000000000000000000000000000000000000000000000002FFF49
:3C3F4800020000000000000000000000000000000000000000000000000000000000000000000000000000000000000000000000000000000000000000002FFF0D
:3C3F8400000000000000000000000000000000000000000000000000000000000000000000000000000000000000000000000000000000000000000000000FFFF3
:3C3FC000000000000000000000000000000000000000000000000000000000000000000000000000000000000000000000000000000000000000000000000FFFB7
:3C3FFC00000000000000000000000000000000000000000000000000000000000000000000000000000000000000000000000000000000000000000000000FFF7B
:3C403800000000000000000000000000000000000000000000000000000000000000000000000000000000000000000000000000000000000000000000001EFE30
:3C407400000000000000000000000000000000000000000000000000000000000000000000000000000000000000000000000000000000000000000000001EFEF4
:3C40B000020000000000000000000000000000000000000000000000000000000000000000000000000000000000000000000000000000000000000000002FFFA4
:3C40EC00020000000000000000000000000000000000000000000000000000000000000000000000000000000000000000000000000000000000000000002FFF68
:3C412800020000000000000000000000000000000000000000000000000000000000000000000000000000000000000000000000000000000000000000002FFF2B
:3C416400000000000000000000000000000000000000000000000000000000000000000000000000000000000000000000000000000000000000000000000FFF11
:3C41A000000000000000000000000000000000000000000000000000000000000000000000000000000000000000000000000000000000000000000000000FFFD5
:3C41DC00000000000000000000000000000000000000000000000000000000000000000000000000000000000000000000000000000000000000000000000FFF99
:3C421800000000000000000000000000000000000000000000000000000000000000000000000000000000000000000000000000000000000000000000001EFE4E
:3C425400000000000000000000000000000000000000000000000000000000000000000000000000000000000000000000000000000000000000000000001EFE12
:3C429000020000000000000000000000000000000000000000000000000000000000000000000000000000000000000000000000000000000000000000002FFFC2
:3C42CC00020000000000000000000000000000000000000000000000000000000000000000000000000000000000000000000000000000000000000000002FFF86
:3C430800020000000000000000000000000000000000000000000000000000000000000000000000000000000000000000000000000000000000000000002FFF49
:3C434400000000000000000000000000000000000000000000000000000000000000000000000000000000000000000000000000000000000000000000000FFF2F
:3C438000000000000000000000000000000000000000000000000000000000000000000000000000000000000000000000000000000000000000000000000FFFF3
:3C43BC00000000000000000000000000000000000000000000000000000000000000000000000000000000000000000000000000000000000000000000001EFEA9
:3C43F800000000000000000000000000000000000000000000000000000000000000000000000000000000000000000000000000000000000000000000001EFE6D
:3C443400000000000000000000000000000000000000000000000000000000000000000000000000000000000000000000000000000000000000000000001EFE30
:3C447000020000000000000000000000000000000000000000000000000000000000000000000000000000000000000000000000000000000000000000002FFFE0
:3C44AC00020000000000000000000000000000000000000000000000000000000000000000000000000000000000000000000000000000000000000000002FFFA4
:3C44E800000000000000000000000000000000000000000000000000000000000000000000000000000000000000000000000000000000000000000000001EFE7C
:3C452400020000000000000000000000000000000000000000000000000000000000000000000000000000000000000000000000000000000000000000002FFF2B
:3C456000020000000000000000000000000000000000000000000000000000000000000000000000000000000000000000000000000000000000000000002FFFEF
:3C459C00000000000000000000000000000000000000000000000000000000000000000000000000000000000000000000000000000000000000000000000FFFD5
:3C45D800000000000000000000000000000000000000000000000000000000000000000000000000000000000000000000000000000000000000000000001EFE8B
:3C461400000000000000000000000000000000000000000000000000000000000000000000000000000000000000000000000000000000000000000000001EFE4E
:3C465000020000000000000000000000000000000000000000000000000000000000000000000000000000000000000000000000000000000000000000003EFEF0
:3C468C00020000000000000000000000000000000000000000000000000000000000000000000000000000000000000000000000000000000000000000002FFFC2
:3C46C800020000000000000000000000000000000000000000000000000000000000000000000000000000000000000000000000000000000000000000002FFF86
:3C470400000000000000000000000000000000000000000000000000000000000000000000000000000000000000000000000000000000000000000000001EFE5D
:3C474000000000000000000000000000000000000000000000000000000000000000000000000000000000000000000000000000000000000000000000001EFE21
:3C477C00000000000000000000000000000000000000000000000000000000000000000000000000000000000000000000000000000000000000000000000FFFF3
:3C47B800000000000000000000000000000000000000000000000000000000000000000000000000000000000000000000000000000000000000000000001EFEA9
:3C47F400000000000000000000000000000000000000000000000000000000000000000000000000000000000000000000000000000000000000000000001EFE6D
:3C483000020000000000000000000000000000000000000000000000000000000000000000000000000000000000000000000000000000000000000000003EFE0E
:3C486C00020000000000000000000000000000000000000000000000000000000000000000000000000000000000000000000000000000000000000000002FFFE0
:3C48A800020000000000000000000000000000000000000000000000000000000000000000000000000000000000000000000000000000000000000000002FFFA4
:3C48E400000000000000000000000000000000000000000000000000000000000000000000000000000000000000000000000000000000000000000000000FFF8A
:3C492000000000000000000000000000000000000000000000000000000000000000000000000000000000000000000000000000000000000000000000000FFF4D
:3C495C00020000000000000000000000000000000000000000000000000000000000000000000000000000000000000000000000000000000000000000002FFFEF
:3C499800000000000000000000000000000000000000000000000000000000000000000000000000000000000000000000000000000000000000000000001EFEC7
:3C49D400000000000000000000000000000000000000000000000000000000000000000000000000000000000000000000000000000000000000000000001EFE8B
:3C4A1000000000000000000000000000000000000000000000000000000000000000000000000000000000000000000000000000000000000000000000001EFE4E
:3C4A4C00000000000000000000000000000000000000000000000000000000000000000000000000000000000000000000000000000000000000000000001EFE12
:3C4A8800008000800080008000800080008000800080008000800080008000800080008000800080008000800080008000800080008000800080008000009EFE56
:3C4AC400000000000000000000000000000000000000000000000000000000000000000000000000000000000000000000000000000000000000000000001EFE9A
:3C4B0000000000000000000000000000000000000000000000000000000000000000000000000000000000000000000000000000000000000000000000001EFE5D
:3C4B3C00000000000000000000000000000000000000000000000000000000000000000000000000000000000000000000000000000000000000000000001EFE21
:3C4B7800000000000000000000000000000000000000000000000000000000000000000000000000000000000000000000000000000000000000000000001EFEE5
:3C4BB400000000000000000000000000000000000000000000000000000000000000000000000000000000000000000000000000000000000000000000001EFEA9
:3C4BF000000000000000000000000000000000000000000000000000000000000000000000000000000000000000000000000000000000000000000000001EFE6D
:3C4C2C00000000000000000000000000000000000000000000000000000000000000000000000000000000000000000000000000000000000000000000001EFE30
:3C4C6800000000000000000000000000000000000000000000000000000000000000000000000000000000000000000000000000000000000000000000001EFEF4
:3C4CA400000000000000000000000000000000000000000000000000000000000000000000000000000000000000000000000000000000000000000000001EFEB8
:3C4CE000000000000000000000000000000000000000000000000000000000000000000000000000000000000000000000000000000000000000000000001EFE7C
:3C4D1C00000000000000000000000000000000000000000000000000000000000000000000000000000000000000000000000000000000000000000000001EFE3F
:3C4D5800000000000000000000000000000000000000000000000000000000000000000000000000000000000000000000000000000000000000000000001EFE03
:3C4D9400000000000000000000000000000000000000000000000000000000000000000000000000000000000000000000000000000000000000000000001EFEC7
:3C4DD000000000000000000000000000000000000000000000000000000000000000000000000000000000000000000000000000000000000000000000001EFE8B
:3C4E0C00000000000000000000000000000000000000000000000000000000000000000000000000000000000000000000000000000000000000000000001EFE4E
:3C4E4800000000000000000000000000000000000000000000000000000000000000000000000000000000000000000000000000000000000000000000001EFE12
:3C4E8400000000000000000000000000000000000000000000000000000000000000000000000000000000000000000000000000000000000000000000001EFED6
:3C4EC000000000000000000000000000000000000000000000000000000000000000000000000000000000000000000000000000000000000000000000001EFE9A
:3C4EFC00000000000000000000000000000000000000000000000000000000000000000000000000000000000000000000000000000000000000000000001EFE5E
:3C4F3800000000000000000000000000000000000000000000000000000000000000000000000000000000000000000000000000000000000000000000001EFE21
:3C4F7400000000000000000000000000000000000000000000000000000000000000000000000000000000000000000000000000000000000000000000001EFEE5
:3C4FB000000000000000000000000000000000000000000000000000000000000000000000000000000000000000000000000000000000000000000000001EFEA9
:3C4FEC00000000000000000000000000000000000000000000000000000000000000000000000000000000000000000000000000000000000000000000001EFE6D
:3C502800000000000000000000000000000000000000000000000000000000000000000000000000000000000000000000000000000000000000000000001EFE30
:3C506400000000000000000000000000000000000000000000000000000000000000000000000000000000000000000000000000000000000000000000001EFEF4
:3C50A000000000000000000000000000000000000000000000000000000000000000000000000000000000000000000000000000000000000000000000001EFEB8
:3C50DC00000000000000000000000000000000000000000000000000000000000000000000000000000000000000000000000000000000000000000000001EFE7C
:3C511800000000000000000000000000000000000000000000000000000000000000000000000000000000000000000000000000000000000000000000001EFE3F
:3C515400000000000000000000000000000000000000000000000000000000000000000000000000000000000000000000000000000000000000000000001EFE03
:3C519000000000000000000000000000000000000000000000000000000000000000000000000000000000000000000000000000000000000000000000001EFEC7
:3C51CC00000000000000000000000000000000000000000000000000000000000000000000000000000000000000000000000000000000000000000000001EFE8B
:3C520800000000000000000000000000000000000000000000000000000000000000000000000000000000000000000000000000000000000000000000001EFE4E
:3C524400000000000000000000000000000000000000000000000000000000000000000000000000000000000000000000000000000000000000000000001EFE12
:3C528000000000000000000000000000000000000000000000000000000000000000000000000000000000000000000000000000000000000000000000001EFED6
:3C52BC00000000000000000000000000000000000000000000000000000000000000000000000000000000000000000000000000000000000000000000001EFE9A
:3C52F800000000000000000000000000000000000000000000000000000000000000000000000000000000000000000000000000000000000000000000001EFE5E
:3C533400000000000000000000000000000000000000000000000000000000000000000000000000000000000000000000000000000000000000000000001EFE21
:3C537000000000000000000000000000000000000000000000000000000000000000000000000000000000000000000000000000000000000000000000001EFEE5
:3C53AC0000000000000000000000000000000000000000000000000000000000000000000000000000000000000000000000000000000E00000000000000E1FFD7
:3C53E8000000000000000000000000000000000000000000000000000000000000000000000000000000000000000000000000000000060000000000000078FE0D
:3C542400000000000000000000000000000000000000000000000000000000000000000000000000000000000000000000000000008000000000000000009EFE30
:3C54600002000000000000000000000000000000000000000000000000000000000000000000000000000000000000000000000000802000000000000000BCFEB4
:3C549C0002000000000000000000000000000000000000000000000000000000000000000000000000000000000000000000000000800000000000000000AFFFA4
:3C54D800000000000000000000000000000000000000000000000000000000000000000000000000000000000000000000000000000000000000000000000FFF8A
:3C55140002000000000000000000000000000000000000000000000000000000000000000000000000000000000000000000000000800600000000000000C9FF0B
:3C5550000200000000000000000000000000000000000000000000000000000000000000000000000000000000000000000000000000060000000000000049FFCF
:3C558C000200000000000000000000000000000000000000000000000000000000000000000000000000000000000000000000000050060000000000000019FF73
:3C55C8000000000000000000000000000000000000000000000000000000000000000000000000000000000000000000000000000000060000000000000078FE2B
:3C56040000000000000000000000000000000000000000000000000000000000000000000000000000000000000000000000000000800600000000000000F8FEEE
:3C56400002000000000000000000000000000000000000000000000000000000000000000000000000000000000000000000000000800600000000000000D8FED0
:3C567C0002000000000000000000000000000000000000000000000000000000000000000000000000000000000000000000000000800000000000000000AFFFC2
:3C56B800020000000000000000000000000000000000000000000000000000000000000000000000000000000000000000000000000000000000000000002FFF86
:3C56F40002000000000000000000000000000000000000000000000000000000000000000000000000000000000000000000000000800000000000000000BEFE3C
:3C573000020000000000000000000000000000000000000000000000000000000000000000000000000000000000000000000000000000000000000000003EFEFF
:3C576C000000000000000000000000000000000000000000000000000000000000000000000000000000000000000000000000000008060000000000000070FE85
:3C57A8000000000000000000000000000000000000000000000000000000000000000000000000000000000000000000000000000000060000000000000078FE49
:3C57E40000000000000000000000000000000000000000000000000000000000000000000000000000000000000000000000000000800600000000000000F8FE0D
:3C58200002000000000000000000000000000000000000000000000000000000000000000000000000000000000000000000000000C0060000000000000089FFFC
:3C585C0002000000000000000000000000000000000000000000000000000000000000000000000000000000000000000000000000800000000000000000AFFFE0
:3C589800000000000000000000000000000000000000000000000000000000000000000000000000000000000000000000000000000000000000000000001EFEB8
:3C58D40002000000000000000000000000000000000000000000000000000000000000000000000000000000000000000000000000800000000000000000AFFF68
:3C591000020000000000000000000000000000000000000000000000000000000000000000000000000000000000000000000000000000000000000000002FFF2B
:3C594C000200000000000000000000000000000000000000000000000000000000000000000000000000000000000000000000000000060000000000000049FFCF
:3C5988000000000000000000000000000000000000000000000000000000000000000000000000000000000000000000000000000000060000000000000078FE67
:3C59C400000000000000000000000000000000000000000000000000000000000000000000000000000000000000000000000000008000000000000000009EFE8B
:3C5A00000200000000000000000000000000000000000000000000000000000000000000000000000000000000000000000000000080280000000000000034FE8E
:3C5A3C0002000000000000000000000000000000000000000000000000000000000000000000000000000000000000000000000000800000000000000000AFFFFE
:3C5A7800020000000000000000000000000000000000000000000000000000000000000000000000000000000000000000000000000000000000000000002FFFC2
:3C5AB40002000000000000000000000000000000000000000000000000000000000000000000000000000000000000000000000000800600000000000000D8FE58
:3C5AF0000200000000000000000000000000000000000000000000000000000000000000000000000000000000000000000000000000060000000000000058FE1C
:3C5B2C000200000000000000000000000000000000000000000000000000000000000000000000000000000000000000000000008080000000000000000036FE07
:3C5B6800000000000000000000000000000000000000000000000000000000000000000000000000000000000000000000000000000000000000000000001EFEE5
:3C5BA400000000000000000000000000000000000000000000000000000000000000000000000000000000000000000000000000008000000000000000009EFEA9
:3C5BE00002000000000000000000000000000000000000000000000000000000000000000000000000000000000000000000000000A000000000000000008FFF59
:3C5C1C0012000000000000000000000000000000000000000000000000000000000000000000000000000000000000000000000000C10000000000000000FFFF7B
:3C5C58000200000000000000000000000000000000000000000000000000000000000000000000000000000000000000000000000000060000000000000058FEB2
:3C5C940002000000000000000000000000000000000000000000000000000000000000000000000000000000000000000000000000800000000000000000AFFFA4
:3C5CD0000208000000000000000000000000000000000000000000000000000000000000000000000000000000000000000000000000060000000000000041FF48
:3C5D0C0002000000000000000000000000000000000000000000000000000000000000000000000000000000000000000000000000000000000000800400EBFFEB
:3C5D4800000000000000000000000000000000000000000000000000000000000000000000000000000000000000000000000000000000000000000004005AFEC3
:3C5D840000000000000000000000000000000000000000000000000000000000000000000000000000000000000000000000000000000000000000800200BCFEA7
:3C5DC000020000000000000000000000000000000000000000000000000000000000000000000000000000000000000000000000000000000000008002009CFE89
:3C5DFC0002000000000000000000000000000000000000000000000000000000000000000000000000000000000000000000000000000000000000800400EBFFFB
:3C5E3800020000000000000000000000000000000000000000000000000000000000000000000000000000000000000000000000000000000000000002000DFF1E
:3C5E7400020000000000000000000000000000000000000000000000000000000000000000000000000000000000000000000000000000000000000002001CFED4
:3C5EB000020000000000000000000000000000000000000000000000000000000000000000000000000000000000000000000000000000000000000014106AFE28
:3C5EEC00000000000000000000000000000000000000000000000000000000000000000000000000000000000000000000000000000000000000008000008FFF6C
:3C5F2800000000000000000000000000000000000000000000000000000000000000000000000000000000000000000000000000000000000000000000001EFE21
:3C5F640000000000000000000000000000000000000000000000000000000000000000000000000000000000000000000000000000000000000000800600F8FE85
:3C5FA00002000000000000000000000000000000000000000000000000000000000000000000000000000000000000000000000000000000000000800000BEFE87
:3C5FDC0002000000000000000000000000000000000000000000000000000000000000000000000000000000000000000000000000000000000000B000009FFF39
:3C6018000200000000000000000000000000000000000000000000000000000000000000000000000000000000000000000000000000000000000000060049FFFC
:3C6054000000000000000000000000000000000000000000000000000000000000000000000000000000000000000000000000000000000000000000060078FE94
:3C6090000000000000000000000000000000000000000000000000000000000000000000000000000000000000000000000000000000008001000000000086FFCE
:3C60CC0000000000000000000000000000000000000000000000000000000000000000000000000000000000000000000000000000A400000000008000003AFE3C
:3C610800000000000000000000000000000000000000000000000000000000000000000000000000000000000000000000000000000000000000000000001EFE3F
:3C61440000000000000000000000000000000000000000000000000000000000000000000000000000000000000000000000000000000000000000800200BCFEE3
:3C6180000200000000000000000000000000000000000000000000000000000000000000000000000000000000000000000000000080280000000080020087FF31
:3C61BC0002000000000000000000000000000000000000000000000000000000000000000000000000000000000000000000000000040600000000800C0001FF0F
:3C61F80000000000000000000000000000000000000000000000000000000000000000000000000000000000000000000000000000800000000000000200BCFE2F
:3C623400020000000000000000000000000000000000000000000000000000000000000000000000000000000000000000000000008000000000000002008DFF1E
:3C627000020000000000000000000000000000000000000000000000000000000000000000000000000000000000000000000000004000000000000004102BFE73
:3C62AC00000000000000000000000000000000000000000000000000000000000000000000000000000000000000000000000000008000000000008000000FFFA8
:3C62E8000000000000000000000000000000000000000000000000000000000000000000000000000000008000000000000000000000000000000000000096FE66
:3C63240000000000000000000000000000000000000000000000000000000000000000000000000000000000000000000000000000000200000000800600DAFEDD
:3C63600002000000000000000000000000000000000000000000000000000000000000000000000000000000000000000000000000804A00000000800600F6FEBB
:3C639C0002000000000000000000000000000000000000000000000000000000000000000000000000000000000000000000000000000C0000000080060005FF2D
:3C63D800020000000000000000000000000000000000000000000000000000000000000000000000000000000000000000000000000002000000000006006BFF15
:3C641400000000000000000000000000000000000000000000000000000000000000000000000000000000000000000001000000008000000000000000009EFF2E
:3C6450000000000000000000000000000000000000000000000000000000000000000000000000000000008000000080000000000000200000000000000014FEDE
:3C648C0000000000000000000000000000000000000000000000000000000000000000000000000000000000000000000000000080000600000080A00000C9FF66
:3C64C8000000000000000000000000000000000000000000000000000000000000000000000000000000000000000000000000000000060000000000000078FE1C
:3C65040000000000000000000000000000000000000000000000000000000000000000000000000000000000000000000000000000800000000000000600F8FEDF
:3C65400002000000000000000000000000000000000000000000000000000000000000000000000000000000000000000000000000A030000000008016107AFF2E
:3C657C0002000000000000000000000000000000000000000000000000000000000000000000000000000000000000000000000000C1060000000000000099FE83
:3C65B800008000800080008000800080008000800080008000800080008000800080008000800080008000800080008000800080008000800080000000000FFF19
:3C65F400020000000000000000000000000000000000000000000000000000000000000000000000000000000000000000000000000006000000000006003EFE21
:3C66300002000000000000000000000000000000000000000000000000000000000000000000000000000000000000000000000000000600000000800700BEFFE2
:3C666C000000000000000000000000000000000000000000000000000000000000000000000000000000000000000000000000000008000000000000000016FED6
:3C66A800000000000000000000000000000000000000000000000000000000000000000000000000008000000000000000000000002000000000002000009EFE5A
:3C66E400000000000000000000000000000000000000000000000000000000000000000000000000000000000000000000000000000000000000000000001EFE5E
:3C672000000000000000000000000000000000000000000000000000000000000000000000000000000000000000000000000000000000000000000000001EFE21
:3C675C00000000000000000000000000000000000000000000000000000000000000000000000000000000000000000000000000000000000000000000001EFEE5
:3C679800000000000000000000000000000000000000000000000000000000000000000000000000000000000000000000000000000000000000000000001EFEA9
:3C67D400000000000000000000000000000000000000000000000000000000000000000000000000000000000000000000000000000000000000000000001EFE6D
:3C681000000000000000000000000000000000000000000000000000000000000000000000000000000000000000000000000000000000000000000000001EFE30
:3C684C00000000000000000000000000000000000000000000000000000000000000000000000000000000000000000000000000000000000000000000001EFEF4
:3C688800000000000000000000000000000000000000000000000000000000000000000000000000000000000400000000000000002000000000000000003AFE78
:3C68C400000000000000000000000000000000000000000000000000000000000000000000000000000000000000000000000000000000000000000000001EFE7C
:3C690000000000000000000000000000000000000000000000000000000000000000000000000000000000000000000000000000000000000000000000001EFE3F
:3C693C00000000000000000000000000000000000000000000000000000000000000000000000000000000000000000000000000000000000000000000001EFE03
:3C697800000000000000000000000000000000000000000000000000000000000000000000000000000000000000000002000000000100000000000000002CFFB5
:3C69B400000000000000000000000000000000000000000000000000000000000000000000000000000000000000000000000000000000000000000000001EFE8B
:3C69F0000000000000000000000000000000000000000000000000000000000000000000000000000000000000000000000000000800000000001000048052FF7E
:3C6A2C00000000000000000000000000000000000000000000000000000000000000000000000000000000000000000000000000000000000000000000001EFE12
:3C6A6800000000000000000000000000000000000000000000000000000000000000000000000000000000000000000000000000000000000000000000001EFED6
:3C6AA400000000000000000000000000000000000000000000000000000000000000000000000000000000000000000000000000000000000000000000001EFE9A
:3C6AE000000000000000000000000000000000000000000000000000000000000000000000000000000200000000000000000000000000000000000000001CFE5E
:3C6B1C00000000000000000000000000000000000000000000000000000000000000000000000000000000000000000000000000000000000000000000001EFE21
:3C6B5800000000000000000000000000000000000000000000000000000000000000000000000000000000000000000000000000000000000000000000001EFEE5
:3C6B9400000000000000000000000000000000000000000000000000000000000000000000000000000000000000000000000000000000000000000000001EFEA9
:3C6BD000000000000000000000000000000000000000000000000000000000000000000000000000000000000000000000000000000000000000000000001EFE6D
:3C6C0C00000000000000000000000000000000000000000000000000000000000000000000000000000000000000000000000000000000000000000000001EFE30
:3C6C4800000000000000000000000000000000000000000000000000000000000000000000000000000000000000000000000000000000000000000000001EFEF4
:3C6C8400000000000000000000000000000000000000000000000000000000000000000000000000000000000000000000000000000000000000000000001EFEB8
:3C6CC000000000000000000000000000000000000000000000000000000000000000000000000000000000000000000000000000000000000000000000001EFE7C
:3C6CFC00000000000000000000000000000000000000000000000000000000000000000000000000000000000000000000000000000000000000000000001EFE40
:3C6D3800000000000000000000000000000000000000000000000000000000000000000000000000000000000000000000000000000000000000000000001EFE03
:3C6D7400008000000000000000000000000000000000000000000000000000000000000000000000000000000000000000000000000000000000000400009AFEC7
:3C6DB000000000000000000000000000000000000000000000000000000000000000000000000000000000000000000000000000000000000000000000001EFE8B
:3C6DEC00000000000000000000000000000000000000000000000000000000000000000000000000000000000000000000000000001000002000000000002EFE0F
:3C6E2800000000000000000000000000000000000000000000000000000000000000000000000000000000000000000000000000000000000000000000001EFE12
:3C6E6400000000000000000000000000000000000000000000000000000000000000000000000000000000000000000000000000002004000000000000007AFE56
:3C6EA000000000000000000000000000000000000000000000000000000000000000000000000000000000000000000000000000000000000000000000001EFE9A
:3C6EDC00020000000000000000000000000000000000000000000000000000000000000000000000000000000000000000000000000000000000000000002FFF4A
:3C6F1800000000000000000000000000000000000000000000000000000000000000000000000000000000000000000000000000000000000000000000001EFE21
:3C6F5400000000000000000000000000000000000000000000000000000000000000000000000000000000000000000000000000000000000000000000001EFEE5
:3C6F9000000000000000000000000000000000000000000000000000000000000000000000000000000000000000000000000000000000000000000000001EFEA9
:3C6FCC00000000000000000000000000000000000000000000000000000000000000000000000000000000000000000000000000000000000000000000001EFE6D
:3C700800000000000000000000000000000000000000000000000000000000000000000000000000000000000000000000000000000000000000000000001EFE30
:3C704400000000000000000000000000000000000000000000000000000000000000000000000000000000000000000000000000000000000000000000001EFEF4
:3C708000000000000000000000000000000000000000000000000000000000000000000000000000000000000000000000000000000000000000000000001EFEB8
:3C70BC00000000000000000000000000000000000000000000000000000000000000000000000000000000000000000000000000000000000000000000001EFE7C
:3C70F800000000000000000000000000000000000000000000000000000000000000000000000000000000000000000000000000000000000000000000001EFE40
:3C713400000000000000000000000000000000000000000000000000000000000000000000000000000000000000000000000000000000000000000000001EFE03
:3C717000020000000000000000000000000000000000000000000000000000000000000000000000000000000000000000000000000000000000000000002FFFB3
:3C71AC00020000000000000000000000000000000000000000000000000000000000000000000000000000000000000000000000000000000000000000002FFF77
:3C71E800020000000000000000000000000000000000000000000000000000000000000000000000000000000000000000000000000000000000000000003EFE2D
:3C722400000000000000000000000000000000000000000000000000000000000000000000000000000000000000000000000000000000000000000000000FFF20
:3C726000000000000000000000000000000000000000000000000000000000000000000000000000000000000000000000000000000000000000000000000FFFE4
:3C729C00000000000000000000000000000000000000000000000000000000000000000000000000000000000000000000000000000000000000000000001EFE9A
:3C72D800000000000000000000000000000000000000000000000000000000000000000000000000000000000000000000000000000000000000000000001EFE5E
:3C731400000000000000000000000000000000000000000000000000000000000000000000000000000000000000000000000000000000000000000000001EFE21
:3C735000020000000000000000000000000000000000000000000000000000000000000000000000000000000000000000000000000000000000000000002FFFD1
:3C738C00020000000000000000000000000000000000000000000000000000000000000000000000000000000000000000000000000000000000000000002FFF95
:3C73C800020000000000000000000000000000000000000000000000000000000000000000000000000000000000000000000000000000000000000000003EFE4B
:3C740400000000000000000000000000000000000000000000000000000000000000000000000000000000000000000000000000000000000000000000000FFF3E
:3C744000000000000000000000000000000000000000000000000000000000000000000000000000000000000000000000000000000000000000000000000FFF02
:3C747C00000000000000000000000000000000000000000000000000000000000000000000000000000000000000000000000000000000000000000000001EFEB8
:3C74B800000000000000000000000000000000000000000000000000000000000000000000000000000000000000000000000000000000000000000000001EFE7C
:3C74F400000000000000000000000000000000000000000000000000000000000000000000000000000000000000000000000000000000000000000000001EFE40
:3C753000020000000000000000000000000000000000000000000000000000000000000000000000000000000000000000000000000000000000000000002FFFEF
:3C756C00020000000000000000000000000000000000000000000000000000000000000000000000000000000000000000000000000000000000000000002FFFB3
:3C75A800000000000000000000000000000000000000000000000000000000000000000000000000000000000000000000000000000000000000000000001EFE8B
:3C75E400020000000000000000000000000000000000000000000000000000000000000000000000000000000000000000000000000000000000000000002FFF3B
:3C762000020000000000000000000000000000000000000000000000000000000000000000000000000000000000000000000000000000000000000000002FFFFE
:3C765C00000000000000000000000000000000000000000000000000000000000000000000000000000000000000000000000000000000000000000000001EFED6
:3C7698000000000000000000000000000000000000000000000000000000000000000000000000000000000000800000000000000000000000000000000016FE22
:3C76D400000000000000000000000000000000000000000000000000000000000000000000000000000000000000000000000000000000000000000000001EFE5E
:3C771000020000000000000000000000000000000000000000000000000000000000000000000000000000000000000000000000000000000000000000002FFF0D
:3C774C00020000000000000000000000000000000000000000000000000000000000000000000000000000000000000000000000000000000000000000002FFFD1
:3C778800020000000000000000000000000000000000000000000000000000000000000000000000000000000000000000000000000000000000000000003EFE87
:3C77C400000000000000000000000000000000000000000000000000000000000000000000000000000000000000000000000000000000000000000000000FFF7B
:3C7800000000000000000000000000000000000000000000000000000000000000000000000000000000000000800000000000000000000000000000000007FFC6
:3C783C00000000000000000000000000000000000000000000000000000000000000000000000000000000000000000000000000000000000000000000001EFEF4
:3C787800000000000000000000000000000000000000000000000000000000000000000000000000000000000000000000000000000000000000000000001EFEB8
:3C78B400000000000000000000000000000000000000000000000000000000000000000000000000000000000000000000000000000000000000000000001EFE7C
:3C78F000020000000000000000000000000000000000000000000000000000000000000000000000000000000000000000000000000000000000000000002FFF2C
:3C792C00020000000000000000000000000000000000000000000000000000000000000000000000000000000000000000000000000000000000000000002FFFEF
:3C796800020000000000000000000000000000000000000000000000000000000000000000000000000000000000000000000000000000000000000000003EFEA5
:3C79A400000000000000000000000000000000000000000000000000000000000000000000000000000000000000000000000000000000000000000000000FFF99
:3C79E000000000000000000000000000000000000000000000000000000000000000000000000000000000000000000000000000000000000000000000000FFF5D
:3C7A1C0000000000000000000000000000000000000000000000000000000000000000000000000000000000000000000000000000000000000000000028ADFF5A
:3C7A5800000000000000000000000000000000000000000000000000000000000000000000000000000000000000000000000000000000000000000000001EFED6
:3C7A9400000000000000000000000000000000000000000000000000000000000000000000000000000000000000000000000000000000000000000000001EFE9A
:3C7AD000020000000000000000000000000000000000000000000000000000000000000000000000000000000000000000000000000000000000000000002FFF4A
:3C7B0C0002000000000000000000000000000000000000000000000000000000000000000000000000000000000000000000000000000000000000000008AFFF85
:3C7B4800000000000000000000000000000000000000000000000000000000000000000000000000000000000000000000000000000000000000000000000FFFF3
:3C7B8400020000000000000000000000000000000000000000000000000001000000000000000000000001000000000000000000000000000000000000002FFF93
:3C7BC00002000000000000000000000000000000000000000000000000800080010000000000000000800000000000000000000000000000000000000040E2FFE5
:3C7BFC0000000000000000000000000000000000000000000000000000000000000000000000000000000000000000000000000000000000000000840600FCFEC9
:3C7C3800000000000000000000000000000000000000000000000000000000000000000000000000000000000000000000000000000000000000000002003CFED4
:3C7C740000000000000000000000000000000000000000000000000000000000000000000000000000000000000000000000000000000000000000800200BCFE98
:3C7CB00002000000000000000000000000000000000000000000000000000000000000000000000000000000000000000000000000000000000000C012085DFE61
:3C7CEC0002000000000000000000000000000000000000000000000000000000000000000000000000000000000000000000000000000000000000A40C0047FF64
:3C7D2800000000000000000000000000000000000000000000000000000000000000000000000000000000000000000000000000000000000000000002003CFEE3
:3C7D640002000000000000000000000000000000000000000000000001000000000000000000000000000000000000000000000000000000000000800400FBFF62
:3C7DA0000200000000000000000000000000000000000000000000800000000000000000000000000000000000000000000000000000000000000000001027FEF0
:3C7DDC0000000000000000000000000000000000000000000000000000000000000000000000000000000000000000000000000000000000000080800628C3FF7B
:3C7E180000000000000000000000000000000000000000000000000000000000000000000000000000000080000000000000000000000000000000000200B4FEFA
:3C7E540000000000000000000000000000000000000000000000000000000000000000000000000000000000000000000000000000000000000000800200BCFEB6
:3C7E900002000000000000000000000000000000000000000000000000000000000000000000000000000000000000000000000000000000000000A012083DFEBF
:3C7ECC0002000000000000000000000000000000000000000000000000000000000000000000000000000000000000000000000000000000000000A40410CFFEF3
:3C7F0800020000000000000000000000000000000000000000000000000000000000000000000000000000000000000000000000000000000000000002000DFF2D
:3C7F440000000000000000000000000000000000000000000000000000000000000000000000000000000000000000000000000000000000000000800400CBFFB3
:3C7F8000000000000000000000000000000000000000000000000000000000000000000000000000000000800000000000000000000000000000000008505AFF94
:3C7FBC000000000000000000000000000000000000000000000000000000000000000000000000000000000000000000000000000000000000000082062849FF91
:3C7FF800000000000000000000000000000000000000000000000000000000000000000000000000000000000000000000000000000000000000000002003CFE11
:3C80340000000000000000000000000000000000000000000000000000000000000000000000000000000000000000000000000000000000000000800200BCFED4
:3C80700002000000000000000000000000000000000000000000000000000000000000000000000000000000000000000000000000000000000000A012083DFEDD
:3C80AC0002000000000000000000000000000000000000000000000000000000000000000000000000000000000000000000000000000000000000A404508BFE15
:3C80E800028000800080008000800080008000800080008000800080008000800080008000800080008000800080008000800080008000800080008002008DFFCC
:3C812400000000000000000000000000000000000000000000000000000000000000000000000000000000000000000000000000000000000000000004004BFFD1
:3C8160000000000000000000000000000000000000000000000000000000000000000000000000000000000000000000000000000000000000000000080816FEBF
:3C819C00000000000000000000000000000000000000000000000000000000000000000000000000000000000000000000000000000000000000000000001EFE8B
:3C81D8000000000000000000000000000000000000000000000001800000008000000000000000000000000000000000000000000000000000000008000086FFDD
:3C821400000000000000000000000000000000000000000000000000000000000000000000000000000000000000000000000000000000000000000000001EFE12
:3C825000000000000000000000000000000000000000000000000000000000000000000000000000000000000000000000000000000000000000000000001EFED6
:3C828C00000000000000000000000000000000000000000000000000000000000000000000000000000000000000000000000000000000000000000000001EFE9A
:3C82C800000000000000000000000000000000000000000000000000000000000000000000000000000000000000000000000000000000000000000000001EFE5E
:3C8304000000000000000000000000000000000000000000000000000000000000000000000000000000000000800000000000000000000000000000002034FE6B
:3C834000000000000000000000000000000000000000000000000000000000000000000000000000000000000000000000000000000000000000000000001EFEE5
:3C837C00000000000000000000000000000000000000000000000000000000000000000000000000000000000000000000000000000000000000000000001EFEA9
:3C83B800000000000000000000000000000000000000000000000000000000000000000000000000000000000400000000000000000000000000002000003AFE2D
:3C83F400000000000000000000000000000000000000000000000000000000000000000000000000000000000000000000000000000000000000000000001EFE31
:3C843000000000000000000000000000000000000000000000000000000000000000000000000000000000000000000000000000000000000000000000001EFEF4
:3C846C00000000000000000000000000000000000000000000000000000000000000000000000000000000000000000000000000000000000000000000001EFEB8
:3C84A800000000000000000000000000000000000000000000000000000000000000000000000000000000000000000000000000000000000000000000001EFE7C
:3C84E400000000000000000000000000000000000000000000000000000000000000000000000000000000000000000000000000000000000000000000001EFE40
:3C852000000000000000000000000000000000000000000000000000000000000000000000000000000000000000000000000000000000000000000000001EFE03
:3C855C00000000000000000000000000000000000000000000000000000000000000000000000000000000000000000000000000000000000000000000001EFEC7
:3C859800000000000000000000000000000000000000000000000000000000000000000000000000000000000000000000000000000000000000000000001EFE8B
:3C85D400000000000000000000000000000000000000000000000000000000000000000000000000000000000000000000000000000000000000000000001EFE4F
:3C861000000000000000000000000000000000000000000000000000000000000000000000000000000000000000000000000000000000000000000000001EFE12
:3C864C00000000000000000000000000000000000000000000000000000000000000000000000000000000000000000000000000000000000000000000001EFED6
:3C868800000000000000000000000000000000000000000000000000000000000000000000000000000000000000000000000000000000000000000000001EFE9A
:3C86C400000000000000000000000000000000000000000000000000000000000000000000000000000000000000000000000000000000000000000000001EFE5E
:3C8700000000000000000000000000000000000000000000000000000000000000000000000000000000400000000000000000000000000000000002000018FEE5
:3C873C00000000000000000000000000000000000000000000000000000000000000000000000000000000000000000000000000000000000000000000001EFEE5
:3C877800000000000000000000000000000000000000000000000000000000000000000000000000000000000000000000000000000000000000000000001EFEA9
:3C87B400000000000000000000000000000000000000000000000000000000000000000000000000000000000000000000000000000000000000000000045EFE29
:3C87F000000000000000000000000000000000000000000000000000000000000000000000000000000000000000000000000000000000000000000000001EFE31
:3C882C00000000000000000000000000000000000000000000000000000000000000000000000000000000000000000000000000000000000000000000045EFEB0
:3C886800000000000000000000000000000000000000000000000000000000002000000000000000000000000000000000000000000000000000000000102FFE77
:3C88A400000000000000000000000000000000000000000000000000000000000000000000000000000000000000000000000000000000000000000000001EFE7C
:3C88E000000000000000000000000000000000000000000000000000000000000000000000000000000000000000000000000000000000000000000000001EFE40
:3C891C00000000000000000000000000000000000000000000000000000020000000000000000000000000000000000000000000000000000000080000009CFE5D
:3C8958000000000000000000000000000000000000000000000000001000000000000000000000000000000000000000000000000000000000000008000016FFB6
:3C899400000000000000000000000000000000000000000000080000000000000000000000000000000000000000000000000000000000000000000000009EFE03
:3C89D000000000000000000000000000000000000000000000000002000000020000000000000000000000000000000000000000000000000000000000001CFE4D
:3C8A0C0000000000000000000000000000000000000000000000000000000000000000000000000000000000000000000000000000000000000000000028ADFF5A
:3C8A4800000000000000000000000000000000000000000000000000000000000000000000000000000000000000000000000000000000000000000000001EFED6
:3C8A8400000000000000000000000000000000000000000000000000000000000000000000000000000000000000000000000000000000000000000000001EFE9A
:3C8AC000020000000000000000000000000000000000000000000000000000000000000000000000000000000000000000000000000000000000000000002FFF4A
:3C8AFC00020000000000000000000000000000000000000000000000000000000000000000000000000000000000000000000000000000000000000000102FFEFF
:3C8B3800020000000000000000000000000000000000000000000000000000000000000000000000000000000000000000000000000000000000000000002FFFD1
:3C8B7400000000000000000000000000000000000000000000000000000000000000000000000000000000000000000000000000000000000000000000000FFFB7
:3C8BB000000000000000000000000000000000000000000000000000000000000000000000000000000000000000000000000000000000000000000000405AFEF1
:3C8BEC00000000000000000000000000000000000000000000000000000000000000000000000000000000000000000000000000000000000000000000001EFE31
:3C8C2800000000000000000000000000000000000000000000000000000000000000000000000000000000000000000000000000000000000000000000001EFEF4
:3C8C6400000000000000000000000000000000000000000000000000000000000000000000000000000000000000000000000000000000000000000000001EFEB8
:3C8CA000020000000000000000000000000000000000000000000000000000000000000000000000000000000000000000000000000000000000000000002FFF68
:3C8CDC00020000000000000000000000000000000000000000000000000000000000000000000000000000000000000000000000000000000000000000002FFF2C
:3C8D1800000000000000000000000000000000000000000000000000000000000000000000000000000000000000000000000000000000000000000000001EFE03
:3C8D5400020000000000000000000000000000000000000000000000000000000000000000000000000000000000000000000000000000000000000000002FFFB3
:3C8D9000020000000000000000000000000000000000000000000000000000000000000000000000000000000000000000000000000000000000000000002FFF77
:3C8DCC000000000000000000000000000000000000000000000000000000000000000000000000000000000000000000009016000000000000000000002833FE6C
:3C8E08000000000000000000000000000000000000000000000000000000000000000000000000000000000000000000000006000000000000000000000018FE12
:3C8E4400000000000000000000000000000000000000000000000000000000000000000000000000000000000000000000000000000000000000000000001EFED6
:3C8E8000020000000000000000000000000000000000000000000000000000000000000000000000000000000000000000A0200000000000000000000000A5FF50
:3C8EBC00020000000000000000000000000000000000000000000000000000000000000000000000000000000000000000000600000000000000000000506DFEB7
:3C8EF8000000000000000000000000000000000000000000000000000000000000000000000000000000000000000000000006000000000000000000000009FF30
:3C8F340002000000000000000000000000000000000000000000000000000000000000000000000000000000000000000080060000000000000000000000A1FFD9
:3C8F70000200000000000000000000000000000000000000000000000000000000000000000000000000000000000000000006000000000000000000000038FE87
:3C8FAC00020000000000000000000000000000000000000000000000000000000000000000000000000000000000000000D0060000000000000000800228E5FE24
:3C8FE800000000000000000000000000000000000000000000000000000000000000000000000000000000000000000000000600000000000000000002003AFE0D
:3C902400000000000000000000000000000000000000000000000000000000000000000000000000000000000000000000000400000000000000000006007CFE8C
:3C9060000200000000000000000000000000000000000000000000000000000000000000000000000000000000000000008036000000000000000080160427FE5D
:3C909C00020000000000000000000000000000000000000000000000000000000000000000000000000000000000000000100600000000000000000006306DFFDE
:3C90D800020000000000000000000000000000000000000000000000000000000000000000000000000000000000000000000600000000000000000006004FFF00
:3C9114000200000000000000000000000000000000000000000000000000000000000000000000000000000000000000008006000000000000000080040065FFAF
:3C9150000200000000000000000000000000000000000000000000000000000000000000000000000000000000000000004016020000000000000000520078FFC0
:3C918C0000000000000000000000000000000000000000000000000000000000000000000000000000000000000000000080040000000000000000A2060056FE27
:3C91C8000000000000000000000000000000000000000000000000000000000000000000000000000000000000800000000004000000000000000000000012FED7
:3C9204000000000000000000000000000000000000000000000000000000000000000000000000000000000000000000008002000000000000000080060072FEB6
:3C9240000200000000000000000000000000000000000000000000000000000000000000000000000000000000000000008002000000000000000080000025FFCA
:3C927C00020000000000000000000000000000000000000000000000000000000000000000000000000000000000000000800400000000000000008806004DFF56
:3C92B800000000000000000000000000000000000000000000000000000000000000000000000000000000000000000000000200000000000000000000001CFE5E
:3C92F40002000000000000000000000000000000000000000000000000000000000000000000000000000000000000000000020000000000000000800600CBFFEA
:3C9330000200000000000000000000000000000000000000000000000000000000000000000000000000000000800000000034000000000000000020000033FFF9
:3C936C0002000000000000000000000000000000000000000000000000000000000000000000000000000000000000000080000000000000000080C00200DCFE27
:3C93A8000000000000000000000000000000000000000000000000000000000000000000000000000000000000000000000000000000000000000000060078FE0D
:3C93E4000000000000000000000000000000000000000000000000000000000000000000000000000000000000000000008006000000000000000080020032FE15
:3C9420000200000000000000000000000000000000000000000000000000000000000000000000000000000000000000008000000000000000000080101037FFB8
:3C945C0002000000000000000000000000000000000000000000000000000000000000000000000000000000000000000090000000000000000000820800ADFE0D
:3C9498000200000000000000000000000000000000000000000000000000000000000000000000000000000000000000000006000000000000000000000038FE5A
:3C94D40002000000000000000000000000000000000000000000000000000000000000000000000000000000000000000000060000000000000000800600CFFF00
:3C95100002000000000000000000000000000000000000000000000000000000000000000000000000000000000000000020000000000000000000400608ABFF05
:3C954C0000000000000000000000000000000000000000000000000000000000000000000000000000000000000000000080000000000000000080C01200ECFF26
:3C9588000000000000000000000000000000000000000000000000000000000000000000000000000000000000000000000000000000000000000000060078FE2B
:3C95C4000000000000000000000000000000000000000000000000000000000000000000000000000000000000000000008006000000000000000080020032FE33
:3C9600000200000000000000000000000000000000000000000000000000000000000000000000000000000000000000008000000000000000000080001027FEF7
:3C963C00020000000000000000000000000000000000000000000000000000000000000000000000000000000000000000B000000000000000000082000007FEB9
:3C9678000000000000000000000000000000000000000000000000000000000000000000000000000000000000000000000006000000000000000000000018FE9A
:3C96B40002000000000000000000000000000000010001000100000000000000000000000000000000000000000000000000060000000000000000800600CFFF1B
:3C96F0000200000000000000000000000000008000800080000000000000008001000000000000000000000000000000000000000000000000000040960089FFDD
:3C972C0000000000000000000000000000000000000000000000000000000000000000000000000000000000000000000080000000000000000080C00A0074FEC5
:3C9768000000000000000000000000000000000000000000000000000000000000000000000000000000000000000000000000000000000000000000060078FE49
:3C97A4000000000000000000000000000000000000000000000000000000000000000000000000000000000000000000008006000000000000000080020032FE51
:3C97E0000200000000000000000000000000000000000000000000000000000000000000000000000000000000000000008000000000000000000080001027FE16
:3C981C00020000000000000000000000000000000000000000000000000000000000000000000000000000000000000000D000000000000000000082000061FE5D
:3C9858000000000000000000000000000000000000000000000000000000000000000000000000000000000000000000000006000000000000000000000018FEB8
:3C98940002000000000000000000000000000000000001000000000000000000000000000000000000000000000000000000060000000000000000800600DFFF2B
:3C98D00002000000000000000000000000000000008000000000000000000000000000000000000000000000000000000000000000000000000000400E04C9FFC0
:3C990C0000000000000000000000000000000000000000000000000000000000000000000000000000000000000000000080000000000000000080C002284FFFE7
:3C99480000000000000000000000000000000000000000000000000000000000000000000000000000000080000000000000000000000000000000000600F0FE6F
:3C9984000000000000000000000000000000000000000000000000000000000000000000000000000000000000000000008006000000000000000080020032FE6F
:3C99C00002000000000000000000000000000000000000000000000000000000000000000000000000000000000000000080060000000000000000800810A9FEA4
:3C99FC000200000000000000000000000000000000000000000000000000000000000000000000000000000000000000008006000000000000000082101033FFD3
:3C9A38000000000000000000000000000000000000000000000000000000000000000000000000000000000000000000000006000000000000000000000009FFE4
:3C9A740002000000000000000000000000000000000000000000000000000000000000000000000000000000000000000000000000000000000000800600C9FF66
:3C9AB00002000000000000000000000000000000000000000000000000000000000000000000000000000080000000000000000000000000000000400624F2FE9E
:3C9AEC0000000000000000000000000000000000000000000000000000000000000000000000000000000000000000000000000000000000000000A202009EFEFE
:3C9B2800000000000000000000000000000000000000000000000000000000000000000000000000000000000000000000000000000000000000000004005AFEA5
:3C9B640000000000000000000000000000000000000000000000000000000000000000000000000000000000000000000000000000000000000000800600F8FE49
:3C9BA00002000000000000000000000000000000000000000000000000000000000000000000000000000000000000000000000000000000000000801004FFFEF6
:3C9BDC0002000000000000000000000000000000000000000000000000000000000000000000000000000000000000000000080000000000000000880000AFFF0D
:3C9C18000080008000800080008000800080008000800080008000800080008000800080008000800080008000800080000000800080008000800080060070FE1C
:3C9C5400020000000000000000000000000000000000000000000000000000000000000000000000000000000000000000000000000000000000000000002FFFA4
:3C9C9000020000000000000000000000000000000000000000000000000000000000000000000000000000000000000000002000000000000000004056003DFEA5
:3C9CCC000000000000000000000000000000000000000000000000000000000000000000000000000000000000000000008000010000000000000000000096FF46
:3C9D0800000000000000000000000000000000000000000000000080000000000000000000800000010000800000000000080000000000000000000800008EFE02
:3C9D4400000000000000000000000000000000000000000000000000000000000000000000000000000000000000000000000000000000000000000000001EFEC7
:3C9D8000000000000000000000000000000000000000000000000000000000000000000000000000000000000000000000000000000000000000000000001EFE8B
:3C9DBC00000000000000000000000000000000000000000000000000000000000000000000000000000000000000000000000000000000000000000000001EFE4F
:3C9DF800000000000000000000000000000000000000000000000000000000000000000000000000000000000000000000000200000000000000000008801CFE8B
:3C9E340000000000000000000000000000000000000000000000000000000000000000000000000000000000000000000000000000000000000000400180D6FF5C
:3C9E70000000000000000000000000000000000000000000000000000000000000000000000000000000000004000100000000000000000000004008000046FE25
:3C9EAC00000000000000000000000000000000000000000000000000000000000000000000000000000000000000000000000000000000000000000000001EFE5E
:3C9EE800000000000000000000000000000000000000000000000000000000000000000000000000000000000000000000000000000000000000000000000FFF30
:3C9F2400000000000000000000000000000000000000000000000000000000000000000000000000000000000000000000000000000000000000000404005EFE9D
:3C9F6000000000000000000000000000000000000000000000000000000000000000000000000000000000000000000000000000000000000000000000001EFEA9
:3C9F9C00000000000000000000000000000000000000000000000000000000000000000000000000000000000000000000000000000000000000000000001EFE6D
:3C9FD800000000000000000000000000000000000000000000000000000000000000000000000000000000000000000000000000000000000000000000001EFE31
:3CA01400000000000000000000000000000000000000000000000000000000000000000000000000000000000000000000000000000000000000000000001EFEF4
:3CA050000000000000000000000000000000000000000000000000000000000000000000000000000000000000000000008001020000000000000000002086FFAC
:3CA08C00000000000000000000000000000000000000000000000000000000000000000000000000000000000000000000000000000000000000000000001EFE7C
:3CA0C800000000000000000000000000000000000000000000000000000000000000000000000000000000000000000000000000000000000000000000001EFE40
:3CA10400000000000000000000000000000000000000000000000000000000000000000000000000000000000000000000000000000000000000000000001EFE03
:3CA14000000000000000000000000000000000000000000000000002000000000000000000000000000000000000000000000000000000000000000000003CFEA7
:3CA17C000000000000000000000000000000000000000000000000000000000000000000000000080000000000000000000000000000000000000000000096FE0B
:3CA1B800000000000000000000000000000000000000000000000000000000000000000000000000000000000000000000000000000000000000000000001EFE4F
:3CA1F400000000000000000000000000000000000000000000000000000000000000000000000000000000000000000000000000000000000000000000001EFE13
:3CA23000000000000000000000000000000000000000000000000000000000000000000000000000000000000000000000000000000000000000000000001EFED6
:3CA26C00000000000000000000000000000000000000000000000000000000000000000000000000000000000000000000000000000000000000000000001EFE9A
:3CA2A800000000000000000000000000000000000000000000000000000000000000000000000000000000000000000000000000000000000000000000001EFE5E
:3CA2E400000000000000000000000000000000000000000000000000000000000000000000000000000000000000000000000000000000000000000000045EFEDE
:3CA32000000000000000000000000000000000000000000000000000000000000000000000000000000000000000000000000000000000000000000000001EFEE5
:3CA35C00000000000000000000000000000000000000000000000000000000000000000000000000000000000000000000000000000000000000000000001EFEA9
:3CA398000000000000000000000000000000000000002000000000000000000020000000000000000000000000000000000000000000000000000000008085FF45
:3CA3D400000000000000000000000000000000000000000000000000000000000000000000000000000000000000000000000000000000000000000000001EFE31
:3CA41000000000000000000000000000000000000000000000000000000000000000000000000000000000000000000000000000000000000000000000001EFEF4
:3CA44C0000000000000000000000000000000000200000002000000000000000000000000000000000000000000000000000000000000000000000000840F0FE5E
:3CA48800000000000000000000000000000000000000100000000000000000000000000000000000000000000000000000000000000000000000000000101EFE5C
:3CA4C400000000000000000000000000000000000000000000000000000000000000000000000000000000000000000000000000000000000000000000001EFE40
:3CA50000000000000000000000000000000000000000000000000000000000000000000000020000000000020000000000000000000000000000000200001CFEFF
:3CA53C0000000000000000000000000000000000000000000000000000000000000000000000000000000000000000000000000000000000000000000048CBFFD1
:3CA57800000000000000000000000000000000000000000000000000000000000000000000000000000000000000000000000000000000000000000000001EFE8B
:3CA5B400000000000000000000000000000000000000000000000000000000000000000000000000000000000000000000000000000000000000000000001EFE4F
:3CA5F000020000000000000000000000000000000000000000000000000000000000000000000000000000000000000000000000000000000000000000002FFFFF
:3CA62C000200000000000000000000000000000000000000000000000000000000000000000000000000000000000000000000000000000000000000204069FF28
:3CA66800000000000000000000000000000000000000000000000000000000000000000000000000000000000000000000000000000000000000000000000FFFA8
:3CA6A400020000000000000000000000000000000000000000000000000000000000000000000000000000000000000000000000000000000000000000002FFF4A
:3CA6E000020000000000000000000000000000000000000000000000000000000000000000000000000000000000000000000000000000000000000000003EFE00
:3CA71C00000000000000000000000000000000000000000000000000000000000000000000000000000000000081060000000000000000C20600000000009CFF17
:3CA758000000000000000000000000000000000000000000000000000000000000000000000000000000000000000600000000000000000006000000000078FE43
:3CA7940000000000000000000000000000000000000000000000000000000000000000000000000000000000008006000000000000000080000000000000FEFE87
:3CA7D0000200000000000000000000000000000000000000000000000000000000000000000000000000000000C02E0000000000000000805600000000003FFF49
:3CA80C0002000000000000000000000000000000000000000000000000000000000000000000000000000000008000000000000000000081000000000000BFFF4F
:3CA84800000000000000000000000000000000000000000000000000000000000000000000000000000000000000000000000000000000000000000000001EFEB8
:3CA8840002000000000000000000000000000000000000000000000000000000000000000000000000000000008006000000000000000180000000000000CFFEC2
:3CA8C000020000000000000000000000000000000000000000000000000000000000000000000000000000000000060000000000008000400600000000008DFF02
:3CA8FC00000000000000000000000000000000000000000000000000000000000000000000000000000000000000000000000081020000820E0000A806005EFF02
:3CA93800000000000000000000000000000000000000000000000000000000000000000000000000000000000000000000000000020000000600000002001AFEC1
:3CA97400000000000000000000000000000000000000000000000000000000000000000000000000000000000000000000000080020000800600008002001AFE05
:3CA9B0000200000000000000000000000000000000000000000000000000000000000000000000000000000000000000000000A0920000A0200000801204F5FFED
:3CA9EC000200000000000000000000000000000000000000000000000000000000000000000000000000000000000000000000810C000081000000C10C0063FFF0
:3CAA2800000000000000000000000000000000000000000000000000000000000000000000000000000000000000000000000000020000000000000002001CFED4
:3CAA6400020000000000000000000000000000000000000000000000000000000000000000000000000000000000000000000080000000800600008004006DFFBE
:3CAAA000020000000000000000000000000000000000000000000000000000000000000000000000000000000000000000000040260000400000000020002FFF84
:3CAADC000000000000000000000000000000000000000000000000000000000000000000000000000000000000000000000000810200808016000081064883FF54
:3CAB18000000000000000000000000000000000000000000000000000000000000000000000000000000000000000000000000000200000006000000000038FEC3
:3CAB5400000000000000000000000000000000000000000000000000000000000000000000000000000000000000000000000080020000800600008002001AFE23
:3CAB90000200000000000000000000000000000000000000000000000000000000000000000000000000000000000000000000A0920000C0200000A01204B3FF0D
:3CABCC000200000000000000000000000000000000000000000000000000000000000000000000000000000000000000000000C2140000810000008214100FFE41
:3CAC0800000000000000000000000000000000000000000000000000000000000000000000000000000000000000000000000000020000000000000002000DFF00
:3CAC4400020000000000000000000000000000000000000000000000000000000000000000000000000000000000000000000080000000800600008004006DFFDC
:3CAC8000020000000000000000000000000000000000000000000000000000000000000000000000000000000000000000000000268001400000004022409CFF72
:3CACBC00020000000000000000000000000000000000000000000000000000000000000000000000000000000000000000000081020000840600008106002EFE9A
:3CACF800000000000000000000000000000000000000000000000000000000000000000000000000000000000000000000000000020000000000000000003EFEE2
:3CAD3400000000000000000000000000000000000000000000000000000000000000000000000000000000000000000000000080020000800200008002001EFE41
:3CAD70000000000000000000000000000000000000000000000000000000000000000000000000000000000000000000000000A0920000A0120100A01204C7FE47
:3CADAC00020000000000000000000000000000000000000000000000000000000000000000000000000000000000000000000084040000A8040000880400C1FFE9
:3CADE800020000000000000000000000000000000000000000000000000000000000000000000000000000000000000000000000020000000200000002003EFEEB
:3CAE2400000000000000000000000000000000000000000000000000000000000000000000000000000000000000000000000080000000800400008004004FFF1C
:3CAE6000000000000000000000000000000000000000000000000000000000000000000000000000000000000000000000000040360000003200002032006BFF52
:3CAE9C00020000000000000000000000000000000000000000000000000000000000000000000000000000000000000000000000000000810E00008106488BFE91
:3CAED800000000000000000000000000000000000000000000000000000000000000000000000000000000000000000000000000000000000200000000001CFE22
:3CAF140000000000000000000000000000000000000000000000000000000000000000000000000000000000000000000000000000000000000000800200BCFEC5
:3CAF5000000000000000000000000000000000000000000000000000000000000000000000000000000000000000000000000000000000C0220000A0120433FEFC
:3CAF8C0002000000000000000000000000000000000000000000000000000000000000000000000000000000000000000000000000000010080000A4045083FFF5
:3CAFC800020000000000000000000000000000000000000000000000000000000000000000000000000000000000000000000000000000000000000002000DFF3D
:3CB004000000000000000000000000000000000000000000000000000000000000000000000000000000000000000000000000000000008000000080040043FFCA
:3CB040000000000000000000000000000000000000000000000000000000000000000000000000800100000000000000000000000000004006020000121054FE97
:3CB07C00020000000000000000000000000000000000000000000000000000000000000000000000000000000000000000000081060000C21600008106488FFFDA
:3CB0B800000000000000000000000000000000000000000000000000000000000000000000000000000000000000000000000000000000000200000000001CFE40
:3CB0F40000000000000000000000000000000000000000000000000000000000000000000000000000000000000000000000008006000000060000800200D2FE42
:3CB130000000000000000000000000000000000000000000000000000000000000000000000000000000000000000000000000A090000080000200A01204F5FF87
:3CB16C000200000000000000000000000000000000000000000000000000000000000000000000000000000000000000000000B010000010000000841430C7FE48
:3CB1A800020000000000000000000000000000000000000000000000000000000000000000000000000000000000000000000000060000000000000002006DFFF5
:3CB1E400000000000000000000000000000000000100010001000000000001000000000000000000000001000000000000000080040000800400008004000FFF90
:3CB220000000000000000000000000000000008000800080000000000080000000000000000000000080000000000000000000000202004008010040021012FEC3
:3CB25C0000000000000000000000000000000000000000000000000000000000000000000000000000000000000000000000000000000081160000810648B3FE9F
:3CB29800000000000000000000000000000000000000000000000000000000000000000000000000000000000000000000000000000000000200000000001CFE5E
:3CB2D40000000000000000000000000000000000000000000000000000000000000000000000000000000000000000000000000000000000000000800200BCFE02
:3CB31000020000000000000000000000000000000000000000000000000000000000000000000000000000000000000000000000000000C0220000A0120413FE56
:3CB34C0002000000000000000000000000000000000000000000000000000000000000000000000000000000000000000000000000000010000080800C10EBFFAD
:3CB38800000000000000000000000000000000000000000000000000000000000000000000000000000000000000000000000000000000000000000002002DFF5B
:3CB3C4000200000000000000000000000000000000000100000001000100000000000000000000000000000000000000000000000000008000000080040073FED3
:3CB40000020000000000000000000000000000000080000000800080000000000000000000000000000000000000000000000000000000400E040020023098FF53
:3CB43C000200000000000000000000000000000000000000000000000000408006000000000000000000000000000000000000810600008006000081064871FFC0
:3CB478000000000000000000000000000000000000000000000000000000000006000000000000000000008000000000000000000000000006000000000096FE78
:3CB4B400000000000000000000000000000000000000000000000000000000000600000000000000000000000000000000000080060000800000008002005AFE76
:3CB4F000000000000000000000000000000000000000000000000000000000A006000000000000000000000000000000000000A090000080100100A012046BFE9A
:3CB52C0002000000000000000000000000000000000000000000000000000000000000000000000000000000000000000000009008000080000000822400FBFE2A
:3CB56800020000000000000000000000000000000000000000000000000000000000000000000000000000000000000000000000060000000000000002006DFF31
:3CB5A4000000000000000000000000000000000000000000000000000000008000000000000000000000000000000000010000800400008006000080040085FED9
:3CB5E00000000000000000000000000000000000000000000000000000000000000000000000000000800180000000800000004002010000060000200A300CFF00
:3CB61C00000000000000000000000000000000000000000000000000000000000000000000000000000000000000000000000081060000880E000081024817FFF4
:3CB65800000000000000000000000000000000000000000000000000000000000000000000000000000000000000000000000000000000000600000002003AFE76
:3CB694000000000000000000000000000000000000000000000000000000000000000000000000000000000000000000000000800600008000000080060018FED8
:3CB6D0000200000000000000000000000000000000000000000000000000000000000000000000000000000000000000000000A0900000C0060100A0100497FEFC
:3CB70C00020000000000000000000000000000000000000000000000000000000000000000000000000000000000000000000088000000810000008830208FFE91
:3CB748000080008000800080008000800080008000800080008000800080008000800080008000800080008000800080008000800680008000800080060089FF31
:3CB78400020000000000000000000000000000000000000000000000000000000000000000000000000000000000000000000000040000000000000000006FFF15
:3CB7C0000200000000000000000000000000000000000000000000000000008001000000000000000000008001000000000000405200004006000040860032FF7A
:3CB7FC00000000000000000000000000000000000000000000000400000000000000000000000000000000000000000000000000000000000000000000001AFEF5
:3CB838000000000000000000000000000000000000000000000000000000000004800000000000000000000000080000000000200000000800000008000010FE0A
:3CB87400000000000000000000000000000000000000000000000000000000000000000000000000000000000000000000000000000000000000000000001EFE7C
:3CB8B000000000000000000000000000000000000000000000000000000000000000000000000000000000000000000000000000000000000000000000101EFF2F
:3CB8EC00000000000000000000000000000000000000000000000000000000000000000000000000000000000000000000000000000000000000000000001EFE04
:3CB92800000000000000000000000000000000000000000000000000000000000000000000000000000000000000000000000000000000000000000000001EFEC7
:3CB964000000000000000000000000000000000000000000000000000000000004000000000000000000000000000000020000001000000000000000000038FF5A
:3CB9A000000000000000000000000000000000000000000000000000000000000000000000000000000000000000000000000000000000000000000000001EFE4F
:3CB9DC00000000000000000000000000000000000000000000000000000000000000000000000000000000002000000000000000000021042000000000005CFF6F
:3CBA18000000000000000000000000000000000000000000000000000000000000000000000000000000000004000000000000000000008000000001000082FFEC
:3CBA5400000000000000000000000000000000000000000000000000000000000000000000000000000000000000000000000000000500000005000000005FFF4E
:3CBA9000000000000000000000000000000000000000000000000000000000000000000000000000000000000000000000000000000000000000000000001EFE5E
:3CBACC00000000000000000000000000000000000000000000000000000000000000000000000000000000000000000000000000000000000000000000001EFE22
:3CBB08000200000000000000000000000000000000000000000000000000080000000000000000000000020004000000000080000800000008000000000098FECB
:3CBB4400000000000000000000000000000000000000000000000000000000000400000000000000000000000000000000000000000040000000000000001EFE65
:3CBB8000000000000000000000000000000000000000000000000000000000000000000000000000000000000000000000000000000000000000000000001EFE6D
:3CBBBC00000000000000000000000000000000000000000000000000000000000000000000000000000000000000000000000000000000000000000000001EFE31
:3CBBF800000000000000000000000000000000000000000000000000000000000000000000000000000000000000000000000000000000044000000000089EFE29
:3CBC3400000000000000000000000000000000000000000000000000000000000000000000000000000000000000000000000000000000000000000000001EFEB8
:3CBC7000000000000000000000000000000000000000000000000000000000000002000000000000000000000000400000000000000000400000000000201EFEDA
:3CBCAC00000000000000000000000000000000000000000000000000000000000000000000000000000000000000000000000000000000000000000000001EFE40
:3CBCE8000000000000000000000000000000000000000000000000000000000000000000000000008000000000000000000020000000000200000000000096FEEA
:3CBD24000000000000000000000000000000000000000000000000000000000000000000000000000000000000000000000000000010000080008000000006FECF
:3CBD60000000000000000000000000000000000000000000000000000000000000000000000000000000400000000000000000000000000000000002000018FE4F
:3CBD9C00000000000000000000000000000000000000000000000000000000000000000000000000000000000000000000000000000000000000000000001EFE4F
:3CBDD800000000000000000000000000000000000000000000000000000000000000000000000000000000000000000000000000000000000000000000001EFE13
:3CBE1400000000000000000000000000000000000000000000000000000000000000000000000000000000000000000000000000000000000000000000001EFED6
:3CBE50000000000000000000000000000000000020000000000000000000000000000000000000000000000000000000000000000000000000000008000036FE5A
:3CBE8C000000000000000000000000000000000000000000000000000000001000000000000000000000000000000000000000001000000000000100018086FF53
:3CBEC80000000000000000000000000000000000000020000000000000000000000000000000000000000000000000000000000000000000000000000840F0FEE8
:3CBF0400000000000000000000000000000000000000000000000000000000000000000000000000000000000000400000000000000000000000000000005AFE69
:3CBF400000000000000000000000000000000000000008000000000000000000000000000000000000000000000000000000000000000000000000200000BEFEE1
:3CBF7C0000000000000000000000000000000000000000002000000000002000000000000000000000000000000000000000001000000000001008200000BEFE45
:3CBFB800000000000000000000000000000000000000000000001000100000000000000000000000000000000000000000000002000000800002008800044EFFD0
:3CBFF400000000000000000000000000000000000000000000000200000000080000000000000000000000000000000000000088020000280100000000008EFFC7
:3CC0300000000000000000000000000000000000000000000000000000000000000000000000000000000000000000000000000204000000000000000082D4FE7A
:3CC06C0000000000000000000000000000000000000000000000000000000000000000000000000000000000000000000000000000000000004800480000DAFE30
:3CC0A80000000000000000000000000000000000000000000000000000000000000000000000000000000000000000000400000000000000008000800000D2FE88
:3CC0E40000000400040004800000008000800480040000000480040000000000000000000000048004800000048004000480040000000000008000800000D6FE98
:3CC12000000000800080000004800400040000000080048000000080048004800480048004800000000004800000008000000080048004800480048000005EFE4F
:3CC15C000000048004800480048004800480048004800480048004800480048004800480048004800480048004800480048004800480048024800488000036FE5F
:3CC1980000000400040004800000008000800480040000000480040000000000000000000000048004800000048004000480040000000000008000800000D6FEE3
:3CC1D400000000800080000004800400040000000080048000000080048004800480048004800000000004800000008000000080048004800480048000005EFE9B
:3CC210000000008000800000048004000400000000800480000000800480048004800480048000000000048000000080000000800480048004200440000094FEC8
:02C24C00FFFFF2
:00000001FF
